:100000000C94A1210C948B300C94B8300C94BE212C
:100010000C94BE210C94BE210C94BE210C94BE21E4
:100020000C94BE210C94BE210C94BE210C945E2431
:100030000C94BE210C94BE210C94BE210C94BE21C4
:100040000C94E5300C94BE210C94BE210C94BE217E
:100050000C94BE210C94BE210C94BE210C94BE21A4
:100060000C94BE210C94BE2177277A277D27802708
:10007000832786278927A927AC27AF27B227B5274B
:10008000B827BB27BE27C127C427C727CA27CD2724
:10009000D027D327D627D927DC27DF270D281028FC
:1000A0001328162819281C281F2822282528282824
:1000B000A928AC28AF28B228B528B828BB28BE2864
:1000C000C128C428C728CA28CD28D028D328D62894
:1000D000D928DC28DF28E228E528E828EB28EE28C4
:1000E000F128F4283229352938293B293E2941298C
:1000F000442947294A294D29502953295629592944
:100100005C295F296229652968296B296E29712973
:10011000742977297A297D296C2A9F2AAE2ABD2A3B
:10012000C62ADB2ADE2AED2AFC2AFF2A0E2B1D2BEB
:10013000202B772C7A2C252D7D2C802C832C862C23
:10014000892C8C2C8F2C922C952C982C9B2C9E2CB3
:10015000A12CA42CA72CAA2CAD2CB02CB32CB62CE3
:10016000B92CBC2CDA2CBF2CC22CC52CC82CCB2C07
:10017000CE2CD12CD42CD72CDA2CDA2CDD2CE02C64
:10018000E32CE62CE92CEC2CEF2CF22CF52CF82CA3
:10019000FB2CFE2C012D042D072D0A2D0D2D102DCD
:1001A000132D162D192D1C2D1F2D222D252D5C2DC7
:1001B000662D702D7A2DA52DC62DD02DDA2DE42D8E
:1001C000EE2DF82D022E132E3E2E692E00D0CC2CB3
:1001D00058A62BF0319B22EAEA51C76C8AB0AB4794
:1001E0001DB34AC2EAAA7CEC660833A7CCB19B21B6
:1001F000CC9C22CBAE8AB0AA8B0C270BD4CD0A3371
:10020000DC2251BB364C710367FF0EB3C113D2EA37
:1002100053C51A0FEBD81513CB7CA46D37C32EF141
:10022000B5A49A2E3B000000000000F0000420332B
:100230002505AA3469549516A832A45E514B205B5B
:10024000A366452E81684D92553905AC2D73649493
:1002500010D2D5AC51515CC29F624CD876099B85B7
:10026000EA994464708FB07B6C91825E6CE189592D
:100270002A93BB8AD82125F3E6AE161900000000A8
:1002800000001E00104C8FB3AFD072733350BF45C7
:1002900047C36B40644E6D0FAF42967D953CFC8228
:1002A000597F59720B3262FB25C923CC48FC972534
:1002B000B738018D5F96549200A3BEC9544A03D249
:1002C000FCD48826252CEBC223899CF1ACF128C9EB
:1002D0000A47382762110000000000003C0030ECA3
:1002E00064C53957F2715264F15C3BC74DCAD4659D
:1002F000231F2F4B3397097DBC64D425D6F2F1938D
:1003000055B1D8D02B484E55E24C8F301A358DB3AD
:100310003C92684C3DCE744BBC53CB5AD121E5DEA8
:1003200032BBC1A80C258BA902CD5261C57D4734D3
:100330000000000000003C00B09CEC3AB942F271B1
:10034000739C946939C7C9B94336651F3797765E80
:10035000B373BC12A6A8D3F6F1522F93553B27488E
:10036000334557148F30E5315CA1D3C26CDA205D80
:100370004E088B1F4633382E2EF982D3201120468B
:1003800003022817020000000000F0000000000037
:1003900000000000000000804A6ACAAC2A262979C1
:1003A00050F1AE88AEB42A54335A87364B65358B3C
:1003B000D3BAE643454449E98632619224AD1C36FE
:1003C0000445E3B6625825B158728A69142572F162
:1003D00029361792AA59AB589C28AB269D627126E4
:1003E000AF9E74F2C585AC6AF6C9975694AAC52724
:1003F0009BDE5033679F6C1843CB5C7CB2A244BA3F
:100400006AF2C9AA32CEAC39272BC62463AA9CBC97
:10041000C960979C7D8ACA525C6276AB0A4B51F3E5
:10042000C9A5AE2C45341AA7AA5357258F5BCA6EAF
:100430004244D44EC93B7731F1D4A5AE32C9D46B16
:100440009F21ABC0CC287D8AA21D3362F4299B0C6E
:10045000CCF0D1A7EC2AD1DD469FB2EBC0301B73A4
:10046000CAAE83426CCCA8AB1209ECAAADAC9264C4
:10047000DC6797AA28E8F07293AA2C612253756969
:10048000A2C4690BD7A1B19237AD1CB9C673CD2CEC
:100490004FD29A115C29426CA99B2276AFCAA31A4B
:1004A0009C28AA27AF6A4926CD9E73EA6504396B5A
:1004B000F6A9A757E4A8D9A71A414823979CBA1BC5
:1004C000668B5A7C9A2ADCC4624E00B44E7140F0AE
:1004D000490A486A4D00968D0B40F815058869B4A5
:1004E000AA9036456DF22943EE12F1C9A70C758C1E
:1004F0003D6B9D32E475CC8E7C8A183631B3F2CADE
:10050000839E268D99A9F0660BD343AB82854A6101
:100510008B453266D35D354EAA0777D70A2BAD9F40
:1005200054C333E2843AF12A5589B5D2E0D6D96270
:10053000E2C9435963CB51278F7952C46F9D3CA6C2
:100540004AD59872B214CA4C7DD149532875C9DA7C
:100550002D0D31D425AB1080264B02486FC1F26AB5
:10056000CD45546A4BBAF5AAD2C4A39932353CEAB8
:100570008CB1AB64B7A87CB6A24DCAABF4E98A567D
:100580002BCDC1A72FC1D4ADCB9CBE0473D7AC7CFF
:10059000C692DD5D72CE194B4C0BF539A72F213C6D
:1005A00034E69CA5F888945C728EEAC24B6DC959FA
:1005B000AA4B2FD52667AD2EBD54D79EB3BAF252A3
:1005C0005D73BA6ACA4A75CD59AA6B2B9135A9CA0F
:1005D0006928DC67912AE4D4D2AE88AAE0C7DCB2ED
:1005E00001AA82C82C33DB000000000000000000DC
:1005F0000F698E8DCD2295B7A97409B2547FC616A6
:1006000083CDB5EF1A7A182297BE75629308E52E4E
:10061000221B0004E09359CB9253CB8C9AAB68D148
:10062000C5C25E9FB2A5220FD972AB5BDFE64E63F7
:10063000A925B04A3BCFAD1FE9AE7A854EF2E5273A
:10064000BFF9CD5FFA4A1C92E3DCE92B35A95A7257
:10065000FF3F0228BDD4ECC1979999AB31A4AC6996
:10066000AEF656978AA6A5245F5D6A96EED676B555
:10067000A9A687FBE6D564BFEAA98B579DE28A87C6
:100680002F59558C6DEEB96494D1759466AB56555F
:10069000C9D9EC8E439D258DB3641143E0E1211946
:1006A000530E61EFCEC8C5B6FC3F08C8461303AB76
:1006B000AE5ECCB36BAFB69910ABBCB3EAE65234C6
:1006C000E2F6AA8A7355D735A6F1DA55C356857670
:1006D000C81063B333B21654C46DF1CA7A5096C8C9
:1006E00025A3E841D1321FCFA256FF0FA989E13CD3
:1006F0003C668F31EB0B2B5FBDA662C6A2ECF16AA4
:10070000AB6BAEF647AB6A31B03C178FAE67438B2D
:100710005A5CC69E182D6B76585A40F198C66A6F7F
:10072000D220BD1B1BE04913037C1366801F3D0CC8
:10073000F05384027E7757C00F660AF8294401BF40
:10074000160BE08F34017C6BF9FFA96B21B922668F
:100750009FAEC7E1707B72BB5BDFEA56BB5C65CBCB
:1007600066C53D67D7AB6D2E643093EEB1CD3D923B
:10077000B99ADAB28E40129A6AEB968F7898B32AB9
:10078000B4D348AA2F7DA77BFB0C73715CCE6E5C43
:10079000526C73799A134B8945E96E4942A957FF08
:1007A0003FA92A4238BA63A6AE0B218D6998FA296F
:1007B00015256A56E9BB53E4CAC5A3EDCA995ADBAD
:1007C000B6B650772DEE1ABA84A224A9ABEB03ED8E
:1007D000D4A4D56E12AAB29C13FD3F01D8413300B8
:1007E000336629A058A3920463EEE593465A98A570
:1007F00014B76D59611656D03565856A5A43B6549B
:1008000064C39501F15AD5857814B46B7527529E4F
:10081000D06DD5836A7B60B75377E66D8EFD4EDB76
:10082000688C07F53B6DA5D911946FF585D5847358
:10083000F63116569326F9C79A594D9AF86B67E622
:1008400035A1E2B75C8977A7AABFF24439ED2A79CE
:10085000CA13D4968AE52D4F705B2A96A7FCC14E29
:10086000B9726EF77B7FA92C79CC6FD2BA8AF5F971
:100870007FC2563C7DDC12DB3E8C89BA4C4A96D353
:100880007595126EBD6FB7BA165A583DB303A614CC
:1008900076C0CC3711C8400422B092D99AC17DF5F8
:1008A000CD6F3E8A3914A572D4286756D489D2B345
:1008B000E9635DD2DA0349A9DBCD473CE3EBBFF442
:1008C0007557ECEE9BF29BBE5634CCA2F2FF0308A8
:1008D000F89155003F091BE09B4803FCE06E80EF58
:1008E000DC1DF0831B02A72855A11A6080A74C4786
:1008F0005C4DA9A6AED9E94AABAAF0E42D23CB768C
:100900002B8337CF6CA4C95FB8EBEA91C43C916AE2
:100910008B531C4AA4A9D742E014A52A5403800093
:10092000CE85082027F7FF070A88294C0225AB4E01
:10093000B4CC6B9E224789F2AA7CEA1ADC3AEDCE4F
:10094000AD6F77873BCF7D9CD5BA75EAE27EB5ABBC
:10095000058D965CE2CE3E3993CA0D03BE37D58035
:10096000053C60010D00029EE7B08000A65E474096
:100970001D4BFF0F0118A9CC0206284EA9143925DA
:10098000694BBA5DAEAA84155AF5BEAB59CF61CE9C
:100990007D6B5B094976EEB51EE5692E44D39AE678
:1009A000277C4D09A547DCF8B9AF7B62B770E6BE7E
:1009B0001A544CB8DDFF0302782D550212B08001A5
:1009C0005E495D4935AE1AD6F69425055B4AD75582
:1009D000943C282DFE7611CAEA06253529024528C1
:1009E0007711D908284E151C501CD3EA6A1449F710
:1009F0004D7B1967534565B1A73E0814A1DC4564DA
:100A0000038000965653C01FAD0278AE0601CBB7E7
:100A1000FF3F08E8589401DF3033E07B6503FC12A8
:100A2000EA805F8B1DF07BA8035E535640A11CAE8D
:100A3000F12CA252DDA43A2BCC718937EA2C335D1C
:100A4000A1CD2A92EC56E736230F7E4B4CD68C3C38
:100A5000DA69355EDDEA68B755A96F1982BD14956C
:100A6000BE61F176C385FB8825E829637387C029B9
:100A70004A55A8060008A094620C20A0A420049463
:100A8000E2F6FF0418CE4D021AD080044691555765
:100A9000076DD9CDAE4F555D5987AEB9D56D5BDBCE
:100AA0007D93B6EDEEE35A6B6AF491D5736B67F5FF
:100AB00047BCD4A79CA534E4D0A6F0E4AAB82DABDB
:100AC000C39B62C2AC74F69FFB720BEC92CDEECF6F
:100AD00043694C5BFF3F0AB89CC400BF681AE03F03
:100AE000F100FC24E9809F2C0D708447A93AD211B3
:100AF000976CA3AAC4D68CB3AC32B31A57E9B2EA46
:100B0000CC7BC2B8EBAA93E871936EAB49AA3B9D2C
:100B1000FBB536A8AD50E9DB8660A75CB44B1A5D27
:100B2000AD54F65DE9363D4A281787CBB40E63DD38
:100B3000ED6E533A5DB8B37B6C5A77E53EEEB3ADDC
:100B4000C5D5F6FC3F0E18A234004B0E2B205BB728
:100B500051A4945AAEA556994B6BBACC5D758E6371
:100B6000D6326735398F5AEB9C3516BF262D4BD6BA
:100B700058ED398DAE5947D31BDCD2669C5DB6C9A2
:100B8000E8EA76379F626D8BCBD342888C2D2A6F33
:100B90008B6A1E36A57CD5B1BB78E2F2564B6EEA65
:100BA0004ECA5B3D87A839096F75E2A66AF7FF0157
:100BB000654AEA3A5CB2CE6E57A748E6D25DBBEC16
:100BC0006217BBDE7D9FDA5C5C7AAAB56ECBD00E75
:100BD000AD6EAFEEF98867BCDC3DAC60B845F3B7ED
:100BE000BFC3DDA2BBABCD898F7FFE1F02F849CC0E
:100BF00000BF873BE0B76003FC9AAA803F921130A8
:100C0000299A0286345F651369E2DA6535598F499E
:100C10005997D5657D29A5DE5697F5858EE45D6DDE
:100C20000E2339DC79D4A5357572EF5195E938E694
:100C3000B94B5D1A266B3B46E014A52A54034001CC
:100C400043BA31607335044E51AA4235FE1F6EAD72
:100C5000CC349C97E823ED5DA4BBF196D9EEFAD491
:100C60004575A6C9E65BDFE60E67AE7CD343FBECB9
:100C70007D9EFDFE7F08D8849901CFB832E0A7148D
:100C800005FC566A8100FC96EA805FCA563E79AA46
:100C9000AAB75E45D3A96AF96415DDB499C69A5519
:100CA000D45062D6B54BD6784B58CD44E014A52A23
:100CB0005403001430853A039EAFF87FA92F122702
:100CC00044DCA6A129180F4D1C8624784534751ADA
:100CD000AAC471D5D8AD2F0ADBCD62AFAE1B330AE3
:100CE0007BBCEA6E4D39E4C9AA9B529592D5ADCD35
:100CF000DCDC4B3E9521CA700F7D1D16A733CAE47C
:100D000091DBBC2C0FA72FEEF0B2DD9DD6A8CBCB8C
:100D100071735A635E2B2632A8ADFA9C193795ACD5
:100D2000E6F7BEDC55D39ADFA9F130496A7EAFDB26
:100D300042798DF94376738A35FF0F04F8C5510166
:100D4000BFA66A400316D0C0CAAB752DCD2537BBF0
:100D5000D9CADA540FEED9296B4730D8E380006A3C
:100D6000266D55EBCA21B9E4D4DD26A5F9E33DB6DD
:100D70007538A3315B9AB6115132D2AA3FFC21CE0D
:100D800022D1D72D9E390B374ED726E1FAC45542D2
:100D9000FD85FB7B7713A3278003D02520010A2044
:100DA0002069D6FF0761CACC385B9AE6A9B6A7ECE2
:100DB0002AC5DD17DFE2E6236B16C32D92CC72B590
:100DC000D5BA86D5ECB994AD9890F47914DE8E53EB
:100DD0003C63230245287711D9008080CF5805F065
:100DE0007B990438C0010A50E0FF0166A9127242E3
:100DF0009B86A51B900E6D76A6262BDCA5CF6D4F8E
:100E0000954DA5BB6E5E45315E6592661445AAB4EC
:100E1000989D5A842A18F69274433AAD5C27DD6D8A
:100E200098A309F592A4654C4DA48256973977C7CB
:100E300068F15DD6DC1D63D44FBEC39D53814EF374
:100E4000899FFFDC5F6692B57AFE7F0248694D0399
:100E500006E834A285954C78A8D29366B1E94D791D
:100E60006F7AD39DF5CC012B860660C5AB08442074
:100E700000CD108DB626118BE83CE6625D3D63F730
:100E800058BB4EF1B02EED28CA74CC9BB8B769A6FA
:100E90000E8F66BEAC48C6ADAEFB9A160EF378FE5A
:100EA000F3BFFFEDFFFF06784A2D005399B52ADB0B
:100EB000628B4C34AA12CBC26CF1188A9EB094CDCE
:100EC0006B2A724A8BBAAC39CB6D29EED2D668AE9A
:100ED000A5A94BD983BBD4C12E6D8FE1CC16B39499
:100EE00023D95339EC53CE5C06FD304BB9725DB457
:100EF000C3DEE9CE65C18EFB86BBACC00A691B9E12
:100F0000D212AAB55378F3336EB14CFF0F0C2830D0
:100F10002C45439A72D8EB9DADBA0B676E7F3D9A14
:100F2000A11DB9F50B02A72855A11A10D65C3A35B8
:100F30002C661AA2757333A7A90F51D254DDB63AA5
:100F4000276A4ACBB6CA92C82C6CED2A7B54D4F2DD
:100F5000D7A31ADE50261EB77A0405997CDCEA195D
:100F60000DA8EB76AB6630A0AA59AD1A4140AA672E
:100F7000A5AA7914AB9EFDFF0C50D6AC9451AB677B
:100F8000609F5AD6B60E69B4AA5293BAE4C5AF06AA
:100F900078C655013FA528E0B7520D18E0B75403B5
:100FA000FC52A6809FCB103845A90AD50030C090CE
:100FB0006E02D85CEDFF0104E8DE1D014BBB126040
:100FC0007A77010CED368AEADDDC64CD2A6A344F8B
:100FD000AD25BB5C55CBE629BD64D7ABA9C53CA408
:100FE000EB885635B6745797BAD8D8DCDD59E97313
:100FF000E394306F6B2CC142C3BAAEBA8514B79C70
:101000005DCE6E49533D6E3A9B4629F3780C28AE6F
:1010100053031A585DD59319B266F5C54C64C89A46
:10102000B1B65896664FC6D55C8BA7BE2E57B3C9CE
:1010300059F166DC3DB7B8D99A72B722A6DEB5D3AE
:10104000D71AB9F4CE46E014A52A5403001430850B
:10105000BA009EAFF87F086848940037300AE00F66
:101060001705FCEE6480DF8B0DF06F8901DE544DB7
:10107000CDB75ECAE265654D8799D99A9557D96E05
:10108000616B5696D584A7AC5E69081B6EB679C4B1
:10109000C16F9648A796447D9EC29D5AD651451869
:1010A0007B31C063C40EF8D524007FB807E077D544
:1010B000D62D114E6A595B57AD70443C1E43D7463E
:1010C000D6F6682C552AC7C4AAB636651CE38FC667
:1010D000D65588962F6E47B1219EF9783C55964695
:1010E000F8AAF25735AC918BD25F794B4AAE66C005
:1010F00067A40AF8C9C400AF382BE035550E30E0BC
:10110000B592FF070A28306C745325B367AC950D70
:101110006324118B5731BCA154AC19F570063CB651
:10112000C60D91A9CE52283632DD9569B2F8D8BAEB
:101130006CDA313469A95330E39274A92A554D927F
:10114000D397AA46132A4DBFEA1E82B174EBEA86F2
:101150000982F6356B18CE1127668D6938479C5C7D
:101160003C96E91CA173F5D8A733A4CEC5E5184178
:10117000913B1FB7730425AA5C53DE1983306C6B57
:101180007A8777E48C3DE51DD150CCB7A66F382720
:1011900076DD12BEA1833878AFF99A0A14B7CFE989
:1011A000BF24445CF2A6FF2276F370937F057C8F08
:1011B000A401016CC8C9801F3CFE1F6E4A9C624A94
:1011C000EB84A508D22E699296AA4833A5699A8B1A
:1011D000248F90A663AAD6429CD7AC3E1BCB525A12
:1011E000B2DAE83AC368CDAA42DEF0E02CAB086D73
:1011F0003583B38C32D4E12AEA3386D89B3A69CF5F
:1012000058736EEAA2DCE3CCD5785273B5333793CA
:1012100048D914AE525C3574120386A8E40007085E
:1012200030D404011A1FFB7F0C78C695013FA52816
:10123000E0B7520B04E0B75407FC5266809FCB4ED8
:1012400056E524A7B63D4515535ABAF554D96D58FD
:10125000EAEA55A7B86EE5ABC798EC8594AD6E4B3E
:10126000B49752B62A6C316C98DB46F3F8B269E653
:101270001BCDE36ABBA92F12AF4BE3C1DE8901434B
:101280005472800314A0C0FF036C657ED3CD1C8B09
:1012900083BA4B37B3C30E5636D9DD61D8759C344B
:1012A000A1AE6B4972DC83D6AEAEDAD6707EB3BA2D
:1012B000EA5CCBE3CE1A9A6BF1B0C76B6EBA39D247
:1012C0005EB5B3DAE4F49CEDDE96C38322B1019EF1
:1012D0007155C04F2906F8ADD40201F82DD501BFD4
:1012E0009419E0E732044E51AA4235001430A41B91
:1012F000033657FB7F0AC8B3C001B9348F3C37B1FE
:10130000284EBBEA34C4B3B8EDAA53E7B032F7AB0A
:10131000CE83D32DDDAF3A17B5D0ECB6AA625246D4
:10132000F34AABAA71699CCAAE4A82BBD8522370F9
:101330008A5215AA01A08021DD18B0B9DAFF030C8A
:10134000C8A33900C5963BA0734F034CADD5B2CCB2
:101350006C42B8CBCA1AE7ACE4B62B9F46C282B641
:10136000AD625A370ADEB68A19DAC169DB2AA62BC2
:101370008590ADAB9CAE0453B6AC72D8122CD9326A
:10138000AAE69AB865CBA8AA6DD4952EA52AB6511F
:101390004FB2A5AAA44559F1FAFF636FC47A1DB5EF
:1013A000ED6137BB6E7562D92DECBF56AD09BA320F
:1013B0008C13C7D6ED4D858699E33EB72986902CD0
:1013C00076DBE69895BB384F5B7229B4516F7DAFE1
:1013D00047B973718C313FE1C9A950D6FDBA27577F
:1013E000C56ECDFDFF02C8D95C032D8AB1304652CF
:1013F000AFBA86261AF6779BD3D51868695963EF7A
:10140000805F5A2D60010B68C003AB6EDE252D177F
:10141000DFFA36BB1D53B16E235DA75D2392B9A7DA
:10142000627F2050847217910D00A080A5330CF0CC
:10143000B327025A4AFD7F6A15715CDC23898DD57A
:1014400036B58C2D36DAC6CCDD915AB9BF51C7CC32
:1014500069766AA612D2B6CEDB6B0FCCBAAA102E72
:10146000BC29ED2AA25BF3A52C2B4FA9259ABCAE73
:10147000BC74D3F070D68AE4C48A3DEE6A9B5735BB
:101480008FD46BE83ED82216AE71F8204D5FB4E6DB
:10149000E183B47CD658460A94F199730947AF2882
:1014A0009D16341CD561A5AA1373654315E271D24C
:1014B000950D6772D84E77B15CCEEEA43C2DBAA4E0
:1014C0005AE5F274576CA9ABFE1F66B7527ACC9DF1
:1014D00084DD4BA936771296C854272C5E1A8A10E1
:1014E000EEB478ABE9D14C4357AFA22757F158B5CA
:1014F000D29182CC73F14A4676B4A8252B1ECD50EA
:10150000BD66AF782426F56EBC63021418D6FA6364
:10151000D3D439E6AABB5736A9C5A76D5ED9AD9716
:101520009CA1B9608B587DC6EE922D7CCB99BB29CE
:10153000D6F2CD7719EBD4255CB6796C3D2669F8E7
:10154000AAB4576314930BD3D9939245AE49F7B01D
:101550008132B938DDCD28E6D4A2F43469D85B8B6A
:10156000C2DBAB907BAD366FEF22A6D5F8FF0166EC
:1015700088823ADDE384314B6C0F4F9C86AAA03DF4
:10158000B5F1EABA3371B559AB1A36554357AF7254
:10159000F8524DDDB2F29192346475A99B318A9470
:1015A0004AA31E3E414A56AFB659C3085FBDBA6A48
:1015B0009CD37C959A9DF2288F0668194CD8CC6CE8
:1015C00039602893005C19D6CA6A9D5C6BD1188A71
:1015D00031C9A84563CB3A382B1795A70495D09904
:1015E0005D9EE25543E77579B3350DCF55EECB5E81
:1015F0002D3836893F073363E98280603508505DB6
:101600002A02AA4DFB7FA54F7AD33C5A8FAEC8A9B8
:1016100070EDBDBA2A3BC3D98F006C4A2140D3CAB2
:101620000818C20401C3861160DA4C055453DA9CD1
:101630005816EDC8EB88E24CECC13623C865D117CB
:10164000BAB420E5E46A8A53A2AC0B7338C9C8B2B5
:1016500068CE9224335B45B1A911B66A754D969850
:10166000C7AAD63791EC12AFC8D1B188972576C0FA
:10167000962201F82E2C015399ADA17A13F57ABD6B
:10168000E6AE43D47DCFBABA0E51F7DDED6AB6941B
:10169000DCF7B4B75A5709DF9DBE62DCD475B7FBDF
:1016A000AA5533E73EE22BDC5D35FC98AF790F0F8E
:1016B000566DBEE1A6AA42CEFF036211BDD8329597
:1016C000AA99D7268FB0AB263E9C2B4D9D1AD57478
:1016D000CA306561744D253298B7360C714BD3BE54
:1016E000EA983ACCADCF2A921F6FB12D2B4F7EAC2A
:1016F000DC36AD38E7D470DFB4E2522C543D5328C9
:10170000B2A4F07257A55EAD83D96423607B9308C1
:101710008C7E441772F3DB869285AD7D571B6B1E62
:10172000A60CFDE52C53315AF3A63B37A16CCDE254
:10173000EE9C8DDD37E9FF03A35BCE18239FAC76CB
:101740007913887CB2AA198C2172F5AA5A50D2B0AA
:10175000D5A97652B253AD952672D51A8DD6DA2414
:10176000C522C25EAB93D6B054A5AB8831CD93925F
:10177000AD3CDB5659F6B6925C836C30EB0A4A5DA1
:10178000C645AF23A853C8C2F2AA243B12D36EEDBC
:10179000F2B30C99DD4B00B6133AE5D4A6AC91E751
:1017A00054C3A4A1E9B6D34E1946A1FD463BB98A5C
:1017B0008EB4294315C2931CBD8C45B08D71BD36C6
:1017C0006DA6A6A2690DF08CAB027E4A31C06FA552
:1017D000161855372EEAFE650C43BB50FA96364E66
:1017E0009382E57BDB3294336EFC19DB74C158B114
:1017F000A6ECCB1743FA9A700C6F6055ABFF1F0A2B
:1018000028306CD4C75419AA9BD5346BCAEE6B56DA
:10181000DDBDA944AC59D508C19CB17A65332472A9
:10182000E7AC958C64E0139557D4BD508D451951A4
:10183000B39861AE64A4CD609485D290474135EAF7
:10184000EA5A734A99A03809C07642A39CDA9435C3
:10185000F28CB166250DDB3C869A4BA035FB984B8C
:1018600072E2B36C6DCB43C847F2A5236F216FCEF4
:10187000168EBC892BB56F38CB32D2966CEE2CDB32
:10188000485BF2B9AB2C112FEE1DEE52072543FB3E
:10189000FF030AD85C4D03258DA9245A52B6228530
:1018A000311FDCD2F2B44CDBE5CAC8520BEEA6C73E
:1018B0002DCF5369436EA5BA94802AAA65FA1C8875
:1018C0003623511BEB30F4B0366BA851243DD6AC17
:1018D000A184444F7FD4E6414670622302A7285575
:1018E000A11A00A08021DD18B0B9DAFF03ACE77EB1
:1018F000C2D41CAB8DC731B5B0AD7691D68D2D71EC
:10190000584D596791B56BC8B23D9CB6ADA1E9E49D
:10191000487EB3DA968D2D6DF5AA7B32D2CCD5AB4D
:10192000EEC9513317AFBA87008B5C3C9BFF0708A9
:1019300088DC950155862AA0857605D4904E003323
:10194000A94719BBB49B7B5B55C8DEE69165552959
:10195000B4A5D9E255E7D01AEEB35797536A78CEBB
:1019600069538A1E1AD5281C598927876D77172530
:101970001E6299113845A90AD50050C0906E0CD846
:101980005C0D815394AA508DFF0769799C4CDCB2A1
:1019900096E5394D43F66A8009281CB0098A011E74
:1019A000461D53D11666FE664CD944A4E99BB1246A
:1019B000DB19265BDA12E38499BE69673493E1B2DE
:1019C000A69DA15418C7DC76855469124DCB154BE2
:1019D000A5B1352D7708592ED138DD4979B56A9DE5
:1019E00074572B916676D3D3BC58AAD9494F566603
:1019F000A51627BDCD8A956A9CF456CB5EA251D21E
:101A00009B5DB15B2C4E5F4916A655FBFF01ADCD2A
:101A1000BE452D5B8FB6C87257DBD4EA0EBC8DACC9
:101A20006BA92790495677A51950C758D2ADA688FB
:101A30002C53DEB2AAA22A2CB8CBA87368B696BCE7
:101A40006348A9305BF2943597802EDE538E1A06D8
:101A500065244F7A6A6E94E13EE96F3E892BF2234A
:101A6000708A5215AA01000A18D28D019BAB217011
:101A70008A5215AAF1FF0ED82E3500CB7578600476
:101A8000A91865F1EA95E46E9C4B79569EAA731CE1
:101A9000751965CCA1B5B8A6D5D99B6452D4D667C3
:101AA0006B92CD71D7904C9B8CAD1953566DDAF675
:101AB000BAAC494BB64A9CB1666F9621CDC69E79A9
:101AC000A79576196712531EDCB59C515EAB6BD798
:101AD000F4077DA56AADC31FCCB788B7717F10B777
:101AE0006A9A36FC89F6BA4B5AF7473913C179CC52
:101AF0005754678AB8F97F0E98A1C401DD288F7406
:101B0000846473AF75EA1A9D2A73F1699A2FB6B28D
:101B1000C7A7AEBA38DB6F9F2AD9928E9ADACA6607
:101B2000295B4A956B129768D15A0678C655013FD2
:101B3000A518E0B7D25126351EAA8B6739AACCAFBB
:101B400044B5CBA80B9909962CADC9642699BBB4B2
:101B500036919E22CE9ABAC4AA1B2C4BEA0B8D0C4E
:101B600023B7FF0F088844C500C5B91AA064B3D1D4
:101B7000A52CA5C56B5697B3BAA76E5963C9AE110C
:101B8000BA652D25995ADAEAB636EB2AE12913B05F
:101B9000AC6B0266D94CC0CCDB0E6841A94DC527A1
:101BA000497BB6B2D6348CADFECB518EB315752DB4
:101BB000571E4ABEDC25DDB909C54A96F0E4C39C30
:101BC000255DDC539E7225A7716F79A969ACF4FF7E
:101BD00001AEE83998BCD68CA219E59898B48A6E03
:101BE00055BCA3D62A9B36F5F259AB6C962A5CED10
:101BF0008C2A2BAD108E93AA6CC595B2A1EB964999
:101C00003333C7A99F2E3342143BA0B9F651265750
:101C10006A4D5946975CA9376C497DB0EA1554B7AF
:101C2000F4C94A9452BDD5149DA6ADAB57DD54A856
:101C30008D6F5E5577CED6BE6A153D285BE5C256E0
:101C40008EAACCE6AD1330725B0266E94EC04A1B29
:101C500009E8A57D152DAA72D8E655B7A026E1ABF7
:101C60005B530D76AAC42975353866E264D4557382
:101C7000A6489C51176D6E1E8DFE1F220B34A2C20A
:101C80009CB08C77970877E256DDD4D2DC499A4332
:101C9000270F576F6DC89D9343F38DAAFA540B5DC0
:101CA000B3AAEE9BB9E4CDC8A66FC2D235239D710D
:101CB000085DD68CBC6761315D5DDA695C482DCD0D
:101CC00068AA0B76F327A32FBA244BD6B4319975A3
:101CD0001FDAD3C6AC2E74B14F198BB8E0A33E65A2
:101CE000CA664D8FFAA439C79658CA9396949A63D8
:101CF000395F58634FCEA5BCFF0F081855CD01D3EF
:101D0000A90560E876079458DEB254D5ADCCCDC8AD
:101D100073D3B0E22DA3CAD5ADDC5EAFAA9A156F1E
:101D200059BDEA1252CB6D3602AA0CE38002BA0901
:101D30002D55C9EA2E5565CC259886E5ECB1D4A081
:101D40009256ABCA56A36055AE44E014A52A54037C
:101D500018D052B0026A0852400B410488DAF0FFF2
:101D60000162578D2DDDD5A53D363677773696DC69
:101D70003825CCDB194BB0D0B0AEA76BDE35CCB676
:101D80009CAA055767DB92AA6AC8827D0BEA3CB71A
:101D9000B0AC8604E8C0AD8D2D8898F59DB10CEFF0
:101DA00024E16BDA3E7D12867F69D7F42D10B6A54B
:101DB0005FE59921112B5ED7EFFF010CF84ECC00A7
:101DC0003FBB1BE0775703FC1512803F4D57D28D68
:101DD000B2B82F5EE9F0CEE4FE7865231852E5E252
:101DE000948F4A10DD95103845A90AD50004847CEB
:101DF000820055DD5A164D87156F5E4B5615DEB2C3
:101E0000796C59A747DBAA72669D96ED0BC3934C7C
:101E10007857CC0C7FB51C239558FD5973A47A6272
:101E2000F2376EE2666E08F01D91007E7134C01FBD
:101E30002906F8B5D400BF171BE0674305BCEEF2D6
:101E4000FFA54DB2D784BAB42ACA5916DD3ACAC41E
:101E50006785A5DF2A2ACA75E56C2DCF28279CBD8A
:101E600021708A5215AA0190A2AECA5CD5F1CAAB04
:101E700032AFA0CEAB2C3ADC4DBE8CB2380D919C6B
:101E8000D38A6E48C72C6E299A641DB3B8A5AC5C82
:101E900074CC92962A6B7397ACFDFFAA90D5AD5582
:101EA0009DA95694D40A97AB7A399CBB445DE8FD52
:101EB000143D53F7AD095DABD4DDAD3ACB0B2FE943
:101EC000BCEAA2CFBC74D5AAAB1D89D2C7ABAD21E9
:101ED000A9D21F8FB15AA7A97A548EE112BCF2651C
:101EE00038BB678AEE56089CA254856A008003A618
:101EF0005077C0F31504D8CAECFF016E4CB88BB50F
:101F0000DAA67523EA244B1BD60D6902BD5D59364E
:101F1000A249B47665DC88C73196ADA1F18A30D983
:101F2000B2BA2EDBC274CB6A9B294DB335AB6BAE14
:101F3000252D56AFB1F8D4B29C23806A5205D075D6
:101F40002803BA29E50002A72855A11A000A18D2C9
:101F50008D019BAB21708A5215AAF1FF0CF829451F
:101F600001BF955A2000BFA53AE0973203FC5C56AA
:101F7000F26A2A202CF9C88A2FC195EC23CD319919
:101F800097B38F34BB125AF11EF2E442A5C8A99848
:101F90009C49D508376D29265552BAB6B558170F42
:101FA0007FDDCE6C5DC2F3D7789A4951B3CEE5ABF5
:101FB0003AD9CC7695BFDB7615F667805F530CF087
:101FC0006BB2037E4E37C06F660AF8ABD9007FA6AE
:101FD00029E0B792FF070AA8BAB814DD9C9298EBE3
:101FE0005554DDA6619D57DB78BBA66E5E6DE36E32
:101FF00099DCB8745589AF70F4D46745DD6C7655BB
:10200000194446B13932C0B0C50E18B65301C19853
:10201000942A144B09C9B2AA682A3DD8FB2A93987E
:102020007663EFA7CC6C3A8DB3AE2AB1ED64C932BA
:10203000EA82674A286B6B33A96994ACBD2D43D4FF
:10204000DD019A2F4C59C938AADFFF07662B2ECC29
:102050009812BBA34B7713B75D8E6A5C43ADF5EA6C
:10206000723077ABD9AB293E2CAC16AFA6F8B4B41E
:102070005ABCEA9ADCCABAF6A86B110FEB50089C5E
:10208000A254856A8001660C56C089A5069821B9BC
:102090004DCD2B6AFBA63637EFC4ED7BDAD6ACB359
:1020A000B4F6697BB52E56D2BB1CD984454AD3728F
:1020B00066551E2EF1CAD5945B989A297717AEE122
:1020C0001C253D4DA6858B99FF07AB1FC1C9336702
:1020D000AD7A9A649D98B58AE18B357DD6CABA09E6
:1020E0008E8CD92BED8ED3D413AFA4194A3773B588
:1020F00092AAA8CCD4754BB3A07609D72D4F82CB2A
:10210000C2138F625812B54AE580C258563F63B970
:1021100030EB597D0B2A12BE7A0DDD8652D8D6B52A
:10212000769DC6A15BD63675B804F72D47B3E4A5F6
:1021300066B79C45B29758D47215C5D6A271EB1DEF
:10214000EEAAB13C5C4D789AC6080F25FF0F0A280D
:1021500030AC3543858958DE5167ED6EAEAB579D87
:10216000448726771D4DA25316EC6D36A5F775D41E
:1021700093BCB525B4E64CCE9AB6509B2AA95F3ADB
:10218000E27069C73E698BD3B903FB862BD5C46C5B
:10219000F6939E5C12AAC46F7AF234F256BFE9C974
:1021A000CD30CAFCA5271765ADE813DEEC44C36348
:1021B000B3799315F1C8D5E9BB24445CF2A6FF229C
:1021C00076F37093FFF47F1F61C2CC14F03C92064B
:1021D000FE1F0AD85C4D0323A8D6342C1AADAA845E
:1021E000B4485FB29AAADBBD75CD6A9A6D8DB6D53B
:1021F000AB69A5A83C1A81026A2833C04BE50E786A
:10220000CE4C01AF86A7E259379670D3CA6E9DD4E3
:10221000ED4DABBA36D48A37AD1C4ED1AB16B77282
:102220007881C89A5DCAE115A266512A4650F09895
:10223000C5A1688A79B243A9A27B45318FFDFF0809
:10224000885B4A00396796ACA47011F5B2AA1225D2
:10225000C4ADCBAAAB2CD1B435AD6D22C4C53B0502
:10226000E0593105BC97CC801D1915709249897FC2
:10227000F00C55A7AD2A34535CD6B4B6211F0BEA37
:10228000D2DA8A7CDCA84B6B1BF271C53EADCDA4C3
:10229000CA595AA7AEC18C10C993D64B42C425AFB8
:1022A00002BE4712C0869C0AF8D9FCFF010CF88ECA
:1022B00059007F0629E0374703FC1EE2805F430296
:1022C000F06BB0037E155DC9A4E6E29E65954D9462
:1022D00073E89A55775ACD6E5B577D285587381B22
:1022E00075435D6EE26695454C9859CB55363C1E5C
:1022F000A6AD5AD514466BB0297595186DA62CD588
:102300004560ACB1F3D28CC0C626495B555D08650B
:102310007419654981DADC65942535CA729E569632
:10232000DC2047795A597C231FE709798AC25BBEB2
:102330002A0D25288F57ADFF0761EECA443B63ADD8
:10234000B91967DD6CB5BA168BA46DF36A5A1A9287
:10235000E12DA32A79509636B72AFB453DDC9DBA7C
:102360006407A2393102A72855A11A4080625E0590
:1023700090DBA802726B1F599E14A99669D4B9B15B
:1023800097D9E6D517DB62239BD754D5A8AE6E5EEE
:102390007357A332B279AD4DADEAE8E6B596509CDD
:1023A00061AB0C504DAA01BA0E654037A51C40E048
:1023B00014A52A5403C00043BA29607335044E5152
:1023C000AA4235FE1F0A2830AC655DBA8AD9E651AB
:1023D00055652A6EAB439D8C9986CC42E014A52AA4
:1023E0005403400055A4312099B652C4D252896991
:1023F0004615CBB20F6C19754AC3B1B867B4C5ADF9
:10240000F0519FD19550642B7DD3900B6B87BB020D
:10241000050CAB92809D3A1330D386038A16294D62
:102420006942D1D2BBADA507C950DF749556444768
:10243000F9CA53B65114E5757F9E4AD19227FC79AB
:10244000195A4BDEF0E7AE58E39ECD5F9E6A2967CE
:10245000517FED25EE2AE7FF01A91ACACDDD92AE24
:10246000ACD8166979BDEA624A7CF4F5AAAA2BB108
:10247000B6C7ABAA2EC5DB66AFBAF9146F5BBC86D4
:10248000EE92BD7DD11ABB2BB6F1456B1B3AD93606
:1024900056EDAD1DD336F1FAC27E983308C931AD81
:1024A0006C4F041655AA42350014D09B2B039A1783
:1024B00061402BC608A891E5FF010228C65500DD42
:1024C000A42B60B832050C135C86A2393A556EE82D
:1024D000A3D03396B6ABAF64C68DD6AC36EB0DF752
:1024E000B8BDEA6A5A2263F6AA5A302E9FD9A36C65
:1024F0008EB9A323BB3E08D58D8A6CEE6193A96289
:102500008BBD113845A90AD50030C053660678BE88
:10251000E2FF0163ECC1B02A1E9DA6A746295D7D9E
:10252000EABA024B75D5A8CB135AB255ADCA4B7057
:102530009D37A52AB4C04DEC82C0294A55A8060093
:10254000038277E7000268192EBD7717129CB9CD78
:10255000415DB39BDEB6447D2925FACA1EC2A80F91
:10256000FB6B770A43BEE2A75CA50C788B7E044E1A
:1025700051AA423500400153A82BE0F98AFF07A277
:102580008FDA63B723A6A16AB1CB8E34C6A69DAA03
:10259000B3D2EABB37F28845A36D4634256B973634
:1025A00049EA947012BA2869822B71085E1252555A
:1025B000A50E784EC8014F931BE0E5760634CF2E6A
:1025C000805ECB02D08C531B52E1B088AC6D884545
:1025D0002252D7A4391AE32A4E9A8ECA83ACB96E16
:1025E0003B8B2E0DE3B6E32C3ED5C3F6B4AB99344A
:1025F0004B595DAE2653BD647379AA216B77ABE965
:10260000894AA2251223708A5215AA01000A98420B
:102610005D00CF5730E03B4105FC12A6809FDD14E2
:10262000F08C2B037E4AF97F6D6C6E895B368FA927
:102630009B115AE933A73117B74A47FDC6929A8BC7
:102640002F654B6B1CE4D5D82DAF658D83AD9AB249
:102650009523769358CAD7CEEC57F8D85B3A8B3D82
:10266000C5E77CE9CDBD3086DA862F978238EC133A
:10267000FEE407ED354BF8734EECD23CEE2FCBB9B0
:102680009D3BFF3F0C98D6DC01479A167FFA141346
:102690004AB5EA6A525375F5AA1B9BB4E03EABEE0D
:1026A000A02A93FCACBAF08E11CABD9A62B252A8AD
:1026B00075E992D57492C60218B6C2030698BE4256
:1026C00002A30E7ECC953BAE2986F6305AB5D6E8ED
:1026D00027CCA84EDBA2AD0AE1AA658F3E46459DF8
:1026E0009623C668557592CEE8BC4D4C4E3A93B1D0
:1026F000515725E96C86D3DDE484AB69AC72551281
:10270000AEA228D34251B89B662F753BF10E77D30A
:102710006A699EE8FF0104A84A9D01338C7140025A
:102720001A08714E5C52EA7E672BEBB59882B7EEC1
:1027300064A47D18B2DB1B9B2250847217910D0498
:10274000F0352D2559B957CAE239B4B169B4F2B49C
:102750005B97B0140515916AF42A805F4A2DE00159
:102760000B684003636956C525578DAD2763B17863
:10277000DC8F7E956BE624325B93EED18358EC4D73
:102780007EE3F7FF66AA8C695392C42D2F6B2A74DF
:10279000DA9DB2DDF636ABCE78DA9DB2D59A01DBA2
:1027A0007745A075C5B87159DA31E56A2263DEDA7A
:1027B0009ABBA37568AF7B3EC39D976087E68B4F3E
:1027C000784B76B209AFFEFD7FB09AACB6C2ADCD04
:1027D000A93B9DCE942CB75A65B69B61BA6615C5C8
:1027E000658CF362948950EE22B2015A957CB9ABA4
:1027F0002529555CC2D394B537A90B9B2C4BB9E660
:10280000A18E63CE8353D2FCAEA5169770CD3BD676
:10281000114F30B44FDB463C62E33DF90007CCD4A6
:102820002981B6D53A282D7EDB51FD092CFBCF77C7
:102830007A4A2C9493BCE1A9E10446FDC537FC65B6
:1028400019567296FF070828A64B00555623A09AE2
:102850009912E71218C35D5652ED29ACE9DFD9AEE3
:10286000E718D65A12AC341F02A72855A11A00083F
:10287000D8269401BF9571C00216D0800734C001DC
:102880000EFC3F089CA254856AC0FF03A0DAA2B2E6
:102890003A44559CFAB0BA4672DAD1DBAE47596178
:1028A000ED2879ED45AF5ADF60F43969AB63D93B68
:1028B000D2BC24A5F5B60F80013E6365C05F6312EC
:1028C0009080062420010EFC3F6EF08AB34BEBC6CD
:1028D000AE36A71A3A5453D6DCEC6623DF582643AB
:1028E000B4CDEA745D9446F0963B9D79982675DBED
:1028F000B3D7B6F590A8919FEA9EEEE99B207DCBD9
:10290000FF03E628C4F8449AFBCDAD8D2A4E4ABC9D
:10291000B88CB98AA948ED7287D3743B1AA99D6F08
:10292000B3CA5E8CC37BF2CE5A5E35665A3AAE5558
:10293000EB9A5775A9296BEEB6D54D37EFB55DC546
:102940009584E5A6FC30E0970C0D5840031CA0C010
:10295000FF03A96B21B922669FAEC7E1707B72BBF2
:102960005BDFEA56BB5C65CB66C53D67D7AB6D2EBA
:10297000643093EEB1CD3D92B99ADAB28E40129A9C
:102980006AEB968F7898B32AB4D348AA2F7DA77B99
:10299000FB0C73715CCE6E5C526C73799A134B892D
:1029A00045E96E4942A957FF3F0CE82ED40206982C
:1029B000D2550316687D17E96EBC658C456DA6E996
:1029C00096DDDEF6B6B75E75D493A59C7B57B36EE5
:1029D0007D1219ADDC298D4F93B487D2B6FCDDACE6
:1029E0002256027018CA1826B590D4DE6B29DA2D4B
:1029F00025178D7988D448795DF77475A194A9D18C
:102A0000F2ED9EAA51A6D49E7FED6FFE2BD1C73D5D
:102A100089FAB70D57D3B4F53755372EE6B2D757E5
:102A2000FF0F04C87E5C020AA8624303A7A86243A2
:102A30004B97DCF214C5A79B7AD39537C31E164A71
:102A40006636F35A896ED43055B532B731B5C1699F
:102A50002CE9F7BC961239D4B5FDDA9B0FD190EE74
:102A6000F5E4170245287711D9409E45DD2B3371D7
:102A70007ABA0B13952DF9F97F01D8B6DD012FF441
:102A80003860D5D1914D9784E64B4E36B21067CD64
:102A900019D92C0194F1786633EB79AF7B578736DF
:102AA000AF52089E6BEA5AB77A94734547AC5A9C6A
:102AB000AFFF070AE84ACD01DBB933C0A6540CA426
:102AC00034D9F20A6CBBB3530E5DA6259B6F75CA51
:102AD0006152DC7449A98AC4764DD7B176C055A637
:102AE00065D826995C56ADB92523D57C3296E99BED
:102AF000207DCB3CFA55AE991A30FC4B3CFF1F09A8
:102B0000582A2500CB9F956C142189A978B35BECDA
:102B1000BAB523134697993ED6B92E79C95BD847E3
:102B200041531FC7E19C855422ECFADBDD23934916
:102B3000B8E678FF3F08983193021CE080075AD628
:102B40001C6B782EBDE52D4FDDADABAA6DC9230200
:102B5000564C93000510908931FC3F04A8BE5C00E0
:102B6000DDA511A0FA72027497C601099CA6AB30CC
:102B70000DCE7AEA6A4A3935FBAA8B1BC676F7ABCB
:102B80002E7919CAD5EFCA570814A1DC4564030091
:102B9000C0FF030998DA220137781A2085D1503A0C
:102BA0003311815D5B95D44404769DD5A93AABF091
:102BB000A13EB7BAD5A92BEBCCA03EB7BDC35A3BBB
:102BC000C86967BDFBE867BFCA9DE97408E7CE77AF
:102BD0007806893257D6F1F18F7DFE1FA5EFD650CA
:102BE0003B678FB93B23497F3387310CE922497D0D
:102BF00056DF69AA396D59DD825692DAE5749DA7D0
:102C0000A6D39A53379956A66F4F599D7B892FDDCE
:102C1000C528AA154BA3D6AE8C8AAD543BA7A93BB9
:102C2000B3545D33E6A65CCB75CD5EC6DAA4CAB9F3
:102C300035AE67B84640B628BBF1F6B7B94720B6FF
:102C400028BBFF0F0E383C2D005FB61960A890938B
:102C5000362BE299B34ED97D89852FBED5AD4F3F36
:102C600064ABA43EBAD3599A2E75D5396D6B0A2D33
:102C70003CECE5DD1FFEB0E7FF03E6A81A355DD6A4
:102C80009A354B8C4E6B1AD6A651B2B5EE589A13A4
:102C90004FB5356768263D4D979CBEC9752F6D7B36
:102CA000BB5BDFFA36A7EFBA25DA16DF69AC23057E
:102CB00045F9ACB98FA39720739F54CE1E45C2A28D
:102CC0004E3ED3D53DB179240DD7484C6EE12CDE74
:102CD000FF0F656989C57366DFE98C330E41C6EA6B
:102CE0005BEF7AF5332550E5EA39D7C56E0814C194
:102CF000DD456403008000AE7033C073331A1040AA
:102D00008F2B14F87F0CF85E4C01BF957BC0021628
:102D1000B0C0C8BA364DB72737BBC529BA716DB731
:102D2000B5ABA8CEBDD4DEA6B25AB1346A1DA73564
:102D300037E55AAE6BEED2B6264C37F54DB99A341C
:102D400039B7C6E11E81D8A2ECE6C77FFEFB7F043F
:102D5000F8AD4C0216B0800656355DA82A6DB9CD87
:102D600069BB2B55B52DB7DBFD9C0DD8328A7BBCDA
:102D70000200030CB12E80DFD23520010E60E0FF8F
:102D80000108684E9D021C60C08C6912B0C028AB5F
:102D90008C9CC02DBB38793115A3B6E416B7DCF591
:102DA0006E57DF545B85BED9E35CC6D66DB1A5BF57
:102DB000995B3B5A3009AF2FEDEC31C45CBED63382
:102DC000DDAD8887E2D2F2F4E0162AB2E3631FF9A0
:102DD000F0E7FF010868210D030428CE9203234A7F
:102DE000CAA61CDAADB470ED1964B7D3914551355C
:102DF00089EA66DEEAE0ABD3294F1FFA52F6905219
:102E00003B257FDDCB9D72728C79CB6FFAD2109E01
:102E1000B42CE14F25703ADCBA2F6FC175CBF2FFAD
:102E20000CE82E94014DBA4A4003166869361CE935
:102E3000BAB8E539707284DB51A4A84EA3C977B142
:102E4000CAD652A871ED2A7B4BA6E037B75ADD48A7
:102E50008E94F164CE6D195591BC6ED7AD1EF5AA56
:102E6000777AC67022CDC7F989CFFF0306B85934E7
:102E70000027D6386058D391552DAA659D4FD1B8FB
:102E8000391767BFC5AE5A1DB57A06F6A97D9DD222
:102E90006C55A52675C99BDFFC6E0E633A3470AF86
:102EA0003EFF1F664EA87A8DEDC4B5CD89D4BCA275
:102EB000DBD127BE334CD94F9B4D578A76BEF5A93F
:102EC000AA2E4FD5CDB7D9435B87134C0DA775AB51
:102ED0007B3EE3196F7FA7A7F9D0305B1D9E9A3424
:102EE00044BCB67DFE1F69FB59DD51D5D7B56F0ACD
:102EF00078C052010F50ACF6A81615F27BEA1947BC
:102F0000D064EBAD76B5EBD196246E626D5B1F0A93
:102F1000A7B9C5ABFD1A62F0F0E26C731C73521DC9
:102F200019946FCE7DED6BD982DC48C72E718BBBB7
:102F3000DFFF1FCCA126BB839318CF4AAD2E31ED06
:102F40003CA72426C354F192648B8A98CB2B2E3451
:102F5000532D0E2F57B30C0D3CBC3C4C4BCAF4F018
:102F6000720F6E4953CDCB532D354D0F2F0FD70C0C
:102F70000D3DBCDC4DD3DDC2F072524F579BC3AB4D
:102F800089BD422D0FAF5AD1719155BC2CC53BD88C
:102F900065F28294184E3BC17342323315454F7926
:102FA000526A55A6A3FF07C36C86B3276D0FA748C7
:102FB000994E553CBC2265364DD1F032D3BE34DA41
:102FC000C3EB82E2DA6535AF31F26B9795BC86D8F8
:102FD0006F82A6730BC69E7299CCCB02AD3C9A1041
:102FE00060AB62052C378400A9730000FE1F02B895
:102FF0003A8C01DFA473400147B92F333B735F5311
:103000007CEC9AC563D5D175AE5BFC645C35879169
:10301000F18336B56855C56FDA452D1C2DB73837A5
:103020009F603CBC9A85A32566F78A571CA9675602
:10303000CA5EF0B216B2F189CE8B9225C72B33CF80
:1030400048B199B4F3FF0ED8AEDD030E38A6D20115
:10305000D3B42CAD6A359DB17DDCEEC465D7F17279
:103060004724B319D9D905704049EA0298BE4201F4
:10307000DFA4694000DF95FC3F02E83E8C01DD657E
:103080000860984C063493CE80E6DA9A146BAA470F
:10309000D15E56AA6D56CD78D9A91C670583E1A4E7
:1030A000BA38EE16869BFA60875B186EEE8B1D6E43
:1030B00061B9693665BA8DE5E53E1CE90E969B5B04
:1030C000AB952B586ECEE53A6AF3B835847B05A3F1
:1030D000E336EF9219B486DBB469B4D12A4E659A0F
:1030E00099CE28D985714C186D6747C65E534A9CA6
:1030F000B5E2854526FE7F0C18B69A01C3750960B6
:10310000D80E0930A09BB6A0BBB0AA164E82EBEA3F
:10311000A9FA59499E59239A273B7866AE4A9C9C46
:10312000E099D32ABD7292EFE688E4454D7E982D52
:10313000626737F9A137A76C94E4C71EDC3CA5830E
:103140001F8BEB520E0E7E2E4EC731D279A53A0D53
:10315000D9C4FF0702D82E9C01DBA63360FB3001E7
:10316000EC20128CE4D8CA3296736341398998C135
:103170004D0DEDB02A05370FB4A5AE5CDC36D0831B
:103180002F4A717B03F73859CDED1EB46B1435B758
:103190006B949991D5DC2648774B66711B21DB2D0A
:1031A0008AC96D88FC26283AB721F41FA365BC02A2
:1031B00038BB3D8EF02BE208B734FF0F0E386E257A
:1031C00000A30D3AA037C5A0059E563586AA5E8C91
:1031D000A482B2D774312269AD1CD3C1D0FA282B96
:1031E0002D47C31BC2C4AEC6CD9C48539AFF0FCC1B
:1031F000677542595D3A4F9D3663B759DC305B5C69
:103200002361F3E21CF1F098C34B7D39CA1D2C2FCA
:10321000B715EF7079BCD2467C52E5F14A6AB371BA
:1032200047C32D39344B2335B77A55338F59DCA238
:1032300044B5BC66728B64F5F698C14D42D42762E2
:10324000382F4AB69C8868BCA695F85CA109867799
:1032500091115BFF0FC6C9715AA292142F6E979CF1
:10326000469DDCB04D621B5570DD55BE0E36C13338
:1032700037A9A7511BCF3CA59E44AC3C7D987B52FF
:103280009672654BF61AD9CAF5912DA22A4BF7FF13
:10329000016DFDC65C95D5F5D5027B5DFD512D2AEE
:1032A000E47775A33AB1FA9B5DEF6A55332760D492
:1032B000E2D9CC764E739D7B3FFB59AE550AC17364
:1032C0004DBDEA9D9E1512A06B757EFE1F6AB1A2D0
:1032D000A795D2D8250FA32DB27A1CB3DEE6D4452C
:1032E0006D56CA9A5BDFFAB6BBDBFD1A8A6F2BF309
:1032F000377B194BD32539FAB96F6DEB31C45C1E9E
:10330000F7AD1FE51CA5485C1ED72B5FF9FA7FAD12
:1033100068C9C53256DFFA542D357BF8EA5BDDE625
:103320004C6D04A6C5EAB984B57523374F834011A7
:10333000CA5D44360028A0E6310F68C000BF8D7911
:10334000C00316D00007FE1FA1DEC244C2FC9C6A67
:10335000887009597B8ACA3B3DA4CFCD5696C4A636
:10336000BBF46E59E29DEAE24AD51265BBB3EB515C
:10337000571299C1D96EB7C73135926AC99BC73404
:103380004C12466C99735FDAD29292646CEE6BD9F0
:103390006A22718FCFE52C41D4DD36A53B19F50C9F
:1033A000EE13EFFC9AD785C862EE6DBFFF0766F398
:1033B000D23843B3D82DAC4DBB70B0DBB00E172C58
:1033C00026AED3326CBB32AB1963F7216C9CE5D4CB
:1033D00033B680CB9A9BAF6CE542707FB3B39DEE62
:1033E0007C552B2640D5E2D9F6B14F75AB7B3DCA53
:1033F000354B1398AFA9577EF397BE190B31F3CD18
:10340000FF03A19F9C9472268D76075590783CEB24
:10341000599DA2876076DA728B5336A5642D7B6E38
:10342000B5FA24DC32B1731FFA1C16ABC6CAE0B57C
:10343000DFCDA1D4781BB6539774A721BCE4FF015C
:1034400001D8B6DD012FF43860D5D1914D9784E6CF
:103450004B4E36B21067CD19D92C0194F1786633F2
:10346000EB79AF7B578736AF52089E6BEA5AB77A33
:1034700094734547AC5A9CAFFF076B6ED9346CE62A
:10348000DCF636B7BEF519AA0F2DDA257B195B4D90
:103490009AA2E7B81D23A526712A03FC94E6010F22
:1034A00068400312E0000730F0FFABC8723393BBF3
:1034B000DCEEB6B7B9F568535CA9A64DB36B730AD9
:1034C000CB71D8BBAF7D2F47B6C7F494379DA934D5
:1034D000F8539778FD3F0E98D528021118E9CC468D
:1034E00098F166A7271D219992B6DC7C17AB2CD2E8
:1034F0002D133BEFAA75CE9447D0EE3AC4292F6125
:103500003531A250B6F8CD1FFF0F028826D4006DCA
:1035100096B5B82505896C3DD2E651B3A6F4486747
:1035200009A08CC7339B79CB670E80CAD7BD6AD5FB
:103530007206B4B5BAB7BDAF735DF3918F78FE3F35
:10354000A36DB4BA8DBCADA692EC0EF2B6AB5D8C99
:10355000A2E0EE16F63FCB39CCB1AC91E50C8BBFB7
:10356000B03BD31D2859E2E94F7BF9E7FF0141EE5B
:10357000D1C8B316EFEED4C33559C4E35BDDEA56C8
:10358000BB59ED92CD91B4784F63199E382C9CCEE7
:10359000A5AFF508C7B0C2611E351EF18C57BCD36C
:1035A000DD4D49B8CE0EF734AD16BCF9FF01A9E8E0
:1035B000C5D87316CFE20EB7BBCDA9BB6FF1F0D55E
:1035C000B7BECDEEC65063729858EE735FDBD6621D
:1035D000729858AE7BDDD35E457293D88D873DECF3
:1035E00061CF709658E1A24DE215EFFF07011891E7
:1035F000B9004D914660652DB3B867ED53F414647E
:10360000114B6E798B5BDEF274C3056AE7EA3DEC21
:10361000712F6D1FB1002BDFF4A31DB32460D4E222
:103620007AE52BDFE91E4348A3EBE4FBFF016E5A6A
:10363000C19954B20960492207ECA816805D26C7DB
:10364000D0A39278743E552F216AB1FA56B7BAD5F5
:10365000AD6F7DBB3D8E75B422367F53CF7EB5678F
:10366000966134DB529FF48EDC88E15FF29DEFFFC0
:10367000076B682ED82A37DFFEF6A7AF21BCC41728
:10368000DFFEF667C86AC34D3ADF614D956CA671DF
:103690009EB1369853495EFB5A8E0A7A43D94F3C05
:1036A000C259E0F408F90967033119A2259EFF0FFA
:1036B000AA8D63A8AA66ADB9A8CB08DD7CFB5BDF49
:1036C000FA36B7396DB5A315BAF876BBDFD39ED7F6
:1036D000DA5C49A52DDE7BDB6B7629AFC76DEF3158
:1036E000D85C1EF7BD1EF548E72889E2F2385FF97D
:1036F000FE7F65186D902DD6ECF656B7BCC5AEC7EB
:1037000030A3016D2DCE8B3DDCD63C6176C5259B6B
:1037100008E52E221B0080012B873860E5ED085854
:10372000C00216B0800634408076D3FE1F6E3F295B
:103730008D9895CD3D00AB3895E2D4EB34817AF28B
:1037400051535075EBCE76B6D3958D924899AB77A1
:10375000BECBDD8E7196048C5A3CE739F7AD6EF521
:103760002AD72A85E0B9263EF1F97FAB1B6194DDAB
:10377000D6DCF174DD37B9E7EAD335B31CE1AF6FBE
:1037800077C7B5D4E0569C77DB5A9DEB988C61C027
:1037900030E91AB0800514306DBB062420010E10EC
:1037A000A006B5FF07A2599551BA17F76A95AB382D
:1037B00042E4925DEE6215333B50D6925DAE6AC52F
:1037C00004A85ABCEBDDEC7677BBDFD39EF63297CC
:1037D000BEF5ADEDB33481F99AFF0706983068E481
:1037E0006B84A0E8D3938DEC849E4B6E368A190DC2
:1037F000A8EA71AF7ADFE7B2ADE000D38BEB9E8F22
:103800007CA673E540A85A1CAF78C5DBDFFF0F0428
:10381000F8A5830312B0800722B0C2EE8D457DC9A2
:10382000CA672942F5353BDFF928660D40CFD7B38B
:103830001CCDAC0614B5680E7DEE4BDFD2395B02B1
:1038400044BDCE57BEF29DEE550AC1734D7EF2F3D4
:10385000FFA62FAA055CD68CBCC716705933B2954B
:103860000BC1FDCDCC663AF351AD9800558B67DBAB
:10387000C73ED5ADEE752FE72C4D60BE26DFF18932
:10388000EFFF03652C96AD7B6A9F66E4208D9C73E9
:10389000AB5BDCE296B7BAF56A6628A0CED5BBDB97
:1038A000FD1EE638A736CF9C80518BEB52D7BCFF6C
:1038B0003F8DDC797283931A60E954036C656A80EA
:1038C00029420C3045EA298B30B3E8C867ADD64CA5
:1038D000B36A9FA37A0DADAA75EAA6B96222E2A9DE
:1038E000BB36A70A2BA34EDC22A642ABDA03358BEC
:1038F0008C4CEA8658542D0E903A11B674B70DF0E0
:103900006DFEDEC4C4E82960002E0F9C6C29712A6C
:103910004E779315772AAEC3CE763C92A54478D1E4
:103920006DCF473BB8BB07F65B43916EA9F2654C80
:10393000C99897699FBAE5339CC19A8FCADE700710
:103940009DEEC979E2EDFFFF076EEF4258B66BA717
:103950007D6825CC59B4F61182C86AF11A462E1238
:103960008D37A7EFC9C9A36E9F76D422737FB4EABF
:10397000510B2D62E2A84743D72E29AE4D92AA28BB
:103980005C8BB96AEB2495E3801D933590BA59039B
:1039900045B3751946279698C5651FCD88BC16D7BF
:1039A0003D3D6310496EEDF8FAEFFF01ABAADEB4BE
:1039B00062669FA27573D36E72B25654CBBAB601CB
:1039C00092C726404B430CC829C501CFB81AE0A7BF
:1039D0001407FC56EA010598605AEAD429B5B8EBF9
:1039E000685317B3966EA32F29545BF68DB5A93291
:1039F0005EDB37B6A1DBB174CB58BA4991F6CDE3A3
:103A00001A3A853A56B76B9862EAF8DCBE9E83D4C0
:103A1000E349F87B7154AFD9E1EF5355B8E7FE3F66
:103A20000488AE8C031208517465E9EC6824594689
:103A30007841D713376D62C35B6FDCD2EA54D2E3AF
:103A400089017E2BF7800714D0E51538608C700350
:103A5000042936BA5E143472F6E8A76F82F42D7327
:103A6000EA473A676AC0F02FF14ECFA88A1CB9D84E
:103A7000FFEE1FBB59D0D6FE3F6E6E5255CDDDA86E
:103A8000AD72559570E3B6E9DDD4844ED9A64B0BE3
:103A900065A52B6D2E4D42B6ACACDB12495DBDF277
:103AA0001E022D6C3530A07246044E51AA423500DC
:103AB000400133493A605AF132966C2C2D5DDA9C04
:103AC00063219FE62F5B294DBC94AFEDA534F172C5
:103AD000B67494BA82C3FECB59469334E52B57E9AA
:103AE000855AE2C7DDE50AA74BA7FF07613D569857
:103AF000D4B6E6A58DC7A801C5DA332C970612D92E
:103B00004FD96D30A665DF794B8B11CFE0AE29CD53
:103B10004E5D38EAF5F464454784CAE65DF59601E2
:103B2000CD976A40031A285DD0DB61EC7DF77B3CC2
:103B30005316DB9AEAF52E6B2D6A4346BCCDB33D96
:103B4000D9B5DA70DF72E794EACD9DDD9DBC73A92B
:103B500028354F1241E196D43D4D24A78A94F8FAB6
:103B6000377CCD767850EAF8FD3F0ED85CCD032B3C
:103B70002AD9D4232BADB426578F58B2B2565C2D18
:103B800063F6CA5A36F5CC592B6B91B5DB42B7BCFC
:103B90005AEA34575DCA62685C55B5ABA3A20913F3
:103BA000A765A82A9853568FA9B23019DDB3A6226B
:103BB000CBA4B4EB18B3EA90922E6D0DBEC3523A6B
:103BC000A723C40A4BD95BAE50323CA473F8420B16
:103BD0003793D5E6F335DD957FABCF87F234DEF74B
:103BE000FF0CF8AD540306F82DD501BF9439E0E77A
:103BF000320BB4AC3B25755FBD8A110D3963F528D6
:103C00004734E0EA4DA31A4991BB568D7A7845D9DD
:103C10007CB29AE19C78E2F169860992B1D7A76EED
:103C20002ED9C75E9FBA84E41C79BDAAD4C4B279E8
:103C3000CDA85397F0A63CA34B53C39AF28C3155B1
:103C40000B1DEAB3F6143D2D35CFD9B31BF3D03E8F
:103C5000EB2C7ADC53368F2BC5D6707FD59E14DBC8
:103C6000C27C55F9724C2FF197E9CF6AB5C27696AE
:103C70003F87D2D258F9FFA2D53938CAECDBA54C20
:103C8000A1985AB9F2D3476FE969CA4EDD89570E38
:103C9000693F4561D995986567256B86644CACF59D
:103CA000E254CD867AD0E6354CD702A57BF6B0A794
:103CB000BDACB5AA541DDBB2F6ECC3D36473D963B3
:103CC000C82CD5DFE90CA133D8F2E6335EEE09B695
:103CD000B254DCF8E7FF010C887E8C02A50A31DDC6
:103CE0005CB2AC265BCF4CEEBBBBDEA7CDA8B475F7
:103CF0004D1CB7D1D528EEE65B767B9A1AC433F318
:103D0000F16D763FE7B6B6EC12919BF28E4011CA88
:103D10005D443680007A2F53402D2414F87F0A2802
:103D200056B9A545558449CC9366D719264B4E966E
:103D3000DD44BAAEBED9CC102842B98BC80660802B
:103D4000F1E9ABCAA623D436DFE18C5574866B9FAC
:103D5000B167BDE1E6BBDB97534588CFAEDFFF031C
:103D60006BC8E2B2423ADFFA16274FAE7DC417B7EE
:103D70002C45AFA4B66D8003D80CF0A79B073CE0A0
:103D800080EBB5113845A90AD50002347565B6A691
:103D9000AEA2346EEA8B9B2413A5ADCDA9C886F3E1
:103DA000CE7E8E6DC9CDB05A7ACFADEEF54C778907
:103DB000833AA9377FE12FAD4887B3FC3F662D02D8
:103DC000624BE38EA5EB10776EB3AA2A2A3974CB27
:103DD0002A0BCBB2E4AEAB4CBCDB9CFAB62A8A29E8
:103DE00033EE93EAA0A6C4B955E892A854A7C46ECE
:103DF0001832CC542DB7B5A9725351BCAAE2532C3A
:103E0000B4F52A8A2BB5D2D5AB28A6D4DA5AAF227C
:103E1000FB322B4BD38A14DCDAC84EA952246B53E5
:103E2000B96AF051B542E931C09BB034A7A6D48538
:103E30006FCA5AC20A2EE66B6789C3B4D82F5D25B4
:103E40000DD352DFF414DF4447FBD25372A21E7528
:103E5000094F898D7CB4E7FF0166313C7C52E3C495
:103E600069F585578651AAD35675A1699D6F7DCA9C
:103E70006A57236DF5CD57D14B50782CDA756946CA
:103E800077B4CEDBB145AD08E52E221B0018D03C3F
:103E900091035A09B18000B213FE7F615A90BAC0F3
:103EA000D7A6690019856ADA9ACD24D9CCCB2A46DF
:103EB0007666F5373B9BC9487B50D48ED9BDA87533
:103EC0006BB362EEF4B8B5ADFDE81BAFCCA2CE7B10
:103ED000D8FB38B3DAC8D055FDA96F7DFF1F06E8BF
:103EE00012D9021268E18C86D4F576C6331AD174E1
:103EF0004A541E6F262B5BDC4293B2ED714D957BCD
:103F00008E53DFBDAEB5B0CC2AEEBBF7762653D9C3
:103F10004A7DFB596E1F2B1B754DBCE313DEA0A61B
:103F200032C8AFFB9318AF207DFF0F615D96493417
:103F3000D20660C7900C8C66F615224D37AA6AC867
:103F40002C6DCD28B2158BE435B3687951E6DA9C37
:103F5000BE154389F0A2DB9577A7A6664977B19A8B
:103F60009E0AD575EBEEF6B0C6E683D2E3EB5ED7DC
:103F7000DA5C48876D9E7BDFF3894011CA5D443669
:103F8000003860EA8C002CB36D0101145F8E81FF54
:103F900007A39DD69932178F668616745FB39AE190
:103FA0004AC4F4CEAE46D11D5A463A99452BAA8250
:103FB000AC0827BE5ADD0C2542BC7BF5D31761F84F
:103FC00096DDEF612CCD8A44C6E3B1571B6269AF21
:103FD000C7999C7B662C6E77F66911F6AABC29A45A
:103FE00087DBE7F4E5141E1AABDD9F627A68ACFA52
:103FF0007F08C84A0C01C57411A0CAEAD1365ADD3F
:1040000046DE565549760779DBC5280AEE6E61FF14
:10401000BDAC0D0245701711D90002E8542D00D532
:104020008405602AB3933567669C6B4E56BD9B6AC8
:10403000DD3959F1AE6EBDF814C5A785E5E253151B
:10404000D59E2E9FCF50E4A607BF596BC53319D814
:10405000A51C89CE94619B747ADD13C44BFCE94E98
:10406000A7AE0AA5CDFF030A88A171158576458AFA
:10407000FF9BDF6C65995CB772DE9DED7277736CA8
:104080004B543563E4A6EEF93457943963E4865F04
:10409000049834DD020E98325D0312E0C0FF030481
:1040A00018B68200D3570860BAF491C65815CA8B67
:1040B000479AFC641AAF19594A9DA1FA6464A9652C
:1040C00086E4E291A7EE9992AB04E0A293040890F3
:1040D0009D33039E7165C04F290AF8ADD402089C38
:1040E000A254856A8000862157C04853011836BC07
:1040F00065A94BAA4B9BD6C4EE11416BDB94EC94A3
:1041000036ED6D4B76939EFCA5EDD94D58EA9ABEDF
:10411000B72BC5764F7F14FED8CD2B7AB2FA9BF21F
:1041200088F0AE0814A1DC45640380008EE030C046
:10413000B253FF0F2B6FB1D9D336DFF636B72685D2
:1041400008E52E221B200025AC2A20CFD352455350
:104150006AA99E4F9B5447B9E4DFC31CC6984565C6
:10416000BB789FCB5CD2EA4367B0E5CD7B389DAD91
:104170002C1537F1FC7F0A28306CADC3A7AA70D785
:10418000D5765D22EE5B57D9F9B8A66D5965169BB9
:10419000A1DE7BD5996DA558DED564115DC269CAD3
:1041A00030255B8532214096260E584A33004BB5A8
:1041B000ADAE9AF030DFB2C7313555E9215DFB3441
:1041C000F6AAC63CA5733FFE1F06D82D2C0133B7B7
:1041D00067A0C5C58DC8B2B79617BF2687F95A9193
:1041E000F3B01F751945CECD71D46554398EDA718F
:1041F000B6D1C530E96E69CB5C518F156649FB803D
:1042000031A2E67D9D55B659D8EA710FDECAE59B0D
:10421000C7D36592556C2EEF304992B13ABDC304B5
:1042200072E7E6F075EBA893ABFF1F02102C34B4D5
:1042300046AFC88ABDD484A9E62DFC461D7B4887BD
:104240002A5F557613E9BA7A97BB9C5569A3AB48A8
:10425000D7D5B10F63F7A1E62A3B8E650CA952555D
:10426000568DB6926A77F1BBC686B23A44FD9CDBA6
:104270005248D738B9EF7BDDC3EE7D67B0F489676C
:10428000BCFE1F63A921B43C16AFB684D20A5FB34B
:10429000AAE2DA32F4CD2A93DF28D727ABC8E25B53
:1042A0009357AFB2D01B0BEEB2CA24AEC3284BA9B2
:1042B0000BAF0E134702A8A64C004D5708A0990C4F
:1042C0000174EDB1EA22BAD4A9CDAA2BEFD6E0BD94
:1042D0006B69AC5A83F7AEB3B16A0BDE32F6A23A21
:1042E000C27973BDF2FDFF0000000700020100006B
:1042F0000304060000000000000000010204081092
:10430000204080010204081020010204081020044B
:10431000040404040404040202020202020303036C
:104320000303030000000023002600290000000012
:1043300000250028002B0000000000240027002A90
:10434000000011241FBECFEFD8E0DEBFCDBF12E0CA
:10435000A0E0B1E0E8E6FBE602C005900D92A837C8
:10436000B107D9F722E0A8E7B2E001C01D92A23D53
:10437000B207E1F70E94A0320C94B2350C94000011
:104380006295262F237384E0289F900111246C7C72
:1043900066956695622B862F8575880F6A7A669575
:1043A000862B0895AF92BF92CF92DF92EF92FF9249
:1043B0000F931F93CF93DF93EC01B62E08811981E1
:1043C000F80164910E94C021E82EF12CFE2CEE240D
:1043D000AA80CB2CD12CC6018A0D911D09973CF0E7
:1043E000F80131966491CE010E94C021E82AC701EC
:1043F0000A2C02C0880F991F0A94E2F720E130E0EE
:104400002C193D0902C0969587952A95E2F72B2D28
:104410002A0D283010F42A8306C028502A830F5F03
:104420001F4F19830883DF91CF911F910F91FF9048
:10443000EF90DF90CF90BF90AF9008952F923F9272
:104440004F925F926F927F928F929F92AF92BF92A4
:10445000CF92DF92EF92FF920F931F93CF93DF9350
:10446000EC018B018B8181111FC061E083E00E9410
:10447000073283E28093B00021E02093B1001092D4
:1044800070001092800089E0809381001092850076
:104490001092840080ED97E09093890080938800CB
:1044A00082E080936F002B83198308831A8230E1A6
:1044B000232E412C44E2542E44EF642E712C3324DD
:1044C000339456E9852E82E00E94C131BC018827D1
:1044D00077FD8095982F1F921F9227E22F932F929E
:1044E00008EEA02E03E0B02EC12CD12CEE24EA94CD
:1044F00013E0F12E00E010E020E030E0A9010E947E
:10450000D3329B01AC01C301B2010E94EB34309362
:1045100089002093880064E0CE010E94D221982E69
:1045200084E00E9476320F900F900F900F90892BAD
:1045300039F0911027C010929B0210929A0270C11C
:1045400082E00E947632892BA1F710929B02109292
:104550009A02109299021092980210929702109269
:104560009602109295021092940210929302109269
:1045700092021092900210928F0210928E021FE00F
:10458000912E4EC18FE0981601F3E92DF0E0E95A23
:10459000FD4F808190E090939B0280939A0261E0AE
:1045A000CE010E94D221182F66E0CE010E94D221B6
:1045B000E82FF0E0E95EFD4F808180939C0284E06B
:1045C0000E947632892B09F062C085E00E94763223
:1045D000892B09F05CC0112309F45BC080919C0217
:1045E000882309F41DC184E00E94C131BC018827E1
:1045F00077FD8095982F1F921F921F923F92AFE3F5
:10460000AA2EB12CC12CD12CEE24EA9413E0F12E69
:1046100000E010E020E030E0A9010E94D332609376
:104620009C0284E00E94C1310F900F900F900F9078
:10463000892B11F410929C0280919C02811124C05C
:1046400083E00E94C131BC01882777FD8095982FB7
:104650001F921F921F921F92EFE0AE2EB12CC12C21
:10466000D12CEE24EA9413E0F12E00E010E020E0DB
:1046700030E0A9010E94D33270939B0260939A02AA
:104680000F900F900F900F904A99ADCFC9C01111A4
:10469000C7C065E0CE010E94D221E82FF0E0EE0F06
:1046A000FF1FE952FE4F8081918190939902809380
:1046B000980265E0CE010E94D221E82FF0E0EE0FD3
:1046C000FF1FE956FE4F808191819093970280935E
:1046D000960264E0CE010E94D221E82FF0E0E95773
:1046E000FE4F80818093950264E0CE010E94D2212A
:1046F000E82FF0E0E958FE4F80818093940280918A
:104700009C02882309F48CC064E0CE010E94D2216F
:10471000E82FF0E0E959FE4F80818093930264E036
:10472000CE010E94D221E82FF0E0E95AFE4F8081AD
:104730008093920264E0CE010E94D221E82FF0E043
:10474000E95BFE4F80818093910263E0CE010E947D
:10475000D221E82FF0E0E15CFE4F8081809390024F
:1047600063E0CE010E94D221E82FF0E0E95CFE4F29
:10477000808180938F0263E0CE010E94D221E82FD6
:10478000F0E0E15DFE4F808180938E0285E00E9423
:1047900076328C0184E00E947632019709F040C0A5
:1047A000012BF1F584E00E94C131BC01882777FD1F
:1047B0008095982F1F921F921F928F92A12CB12C3F
:1047C000650118EEE12E13E0F12E00E010E024E187
:1047D00030E040E050E00E94D3326093930284E0E6
:1047E0000E94C131BC01882777FD8095982F1F92C8
:1047F0001F921F921F9256E9A52EB12CC12CD12CCD
:1048000024E130E040E050E00E94D33260938E0219
:104810008DB79EB708960FB6F8949EBF0FBE8DBF9A
:1048200083E00E94C131BC01882777FD8095982FD5
:104830001F921F921F921F9224E6A22EB12CC12C10
:10484000D12CEE24EA9413E0F12E00E010E020E0F9
:1048500030E0A9010E94D3328B0184E00E947632BD
:104860000F900F900F900F90892B39F485E00E94E4
:104870007632892B11F400E010E0B801882777FD2B
:104880008095982F0E945E319FE099121CCE4C9922
:1048900002C04A9BFECFDF91CF911F910F91FF90F5
:1048A000EF90DF90CF90BF90AF909F908F907F90D0
:1048B0006F905F904F903F902F9008951F920F92AE
:1048C0000FB60F9211242F923F924F925F926F92E8
:1048D0007F928F929F92AF92BF92CF92DF92EF9290
:1048E000FF920F931F932F933F934F935F936F9379
:1048F0007F938F939F93AF93BF93EF93FF93CF9348
:10490000DF93CDB7DEB7A297DEBFCDBF80918D021A
:104910008093B400789490919C02992301F1809146
:104920008C02891720F48F5F80938C0202C0109252
:104930008C02E0918C02E93280F5F0E0EA5FFE4FF4
:10494000A08120919A0230919B02BB27A7FDB095D0
:104950000E942735BB27A92F982F872F20C0809131
:104960000401909105019C013695279580FF03C0B5
:1049700080E098EB02C080E090E028273927309350
:1049800005012093040180919A0290919B0220FDE1
:1049900006C091958195910902C080E090E08090D9
:1049A0008F02992487FC909460908802709089020D
:1049B00060918E0240918A0250918B0264039001B3
:1049C000659F300D1124220F232F221F330BFC0172
:1049D000E21BF30B869CC001879C900D969C900D6A
:1049E0001124880F892F881F990BE81BF90B409021
:1049F0009002552447FC50944091860250918702C2
:104A00005A834983449EC001459E900D549E900D4B
:104A10001124880F892F881F990B1F01281A390A22
:104A200080919102482F552747FD50955C834B8319
:104A300040918402509185025E834D836B817C811D
:104A4000649FC001659F900D749F900D1124880F85
:104A5000892F881F990BA101481B590B58874F8339
:104A600080919202482F552747FD50955A874987D4
:104A700040918202509183025C874B8769857A85D9
:104A8000649FC001659F900D749F900D1124880F45
:104A9000892F881F990B4F815885481B590B5E87BA
:104AA0004D8780919302482F552747FD5095588B8D
:104AB0004F8740918002509181025A8B498B6F85BC
:104AC0007889649FC001659F900D749F900D11249B
:104AD000880F892F881F990B4D855E85481B590BC0
:104AE0005C8B4B8B80919402482F552747FD509546
:104AF0005E8B4D8B40917E0250917F02588F4F8B81
:104B00006D897E89649FC001659F900D749F900D93
:104B10001124880F892F881F990B4B895C89481BAA
:104B2000590B5A8F498F80919502482F552747FD81
:104B300050955C8F4B8F40917C0250917D025E8F2F
:104B40004D8F6B8D7C8D649FC001659F900D749F10
:104B5000900D1124880F892F881F990B498D5A8D2C
:104B6000481B590B58A34F8FA0909602B090970204
:104B7000E0907A02F0907B029501D7010E941035F7
:104B8000AFE09595879577956795AA95D1F76A01D6
:104B9000C61AD70A009198021091990240917802A2
:104BA000509179025AA349A39801DA010E94103565
:104BB000BFE09595879577956795BA95D1F7A6014A
:104BC000461B570B411562E056073CF441157EEF3A
:104BD00057072CF440E05EEF02C04FEF51E08E9E8D
:104BE000C0018F9E900D9E9E900D1124880F892FDD
:104BF000881F990B860D971D90938B0280938A02D4
:104C0000429CC001439C900D529C900D1124880F32
:104C1000892F881F990BE981FA818E0F9F1F90932E
:104C2000890280938802EB81FC812F813885E29F85
:104C3000C001E39F900DF29F900D1124880F892FE2
:104C4000881F990BED81FE818E0F9F1F9093870225
:104C500080938602E985FA852D853E85E29FC00115
:104C6000E39F900DF29F900D1124880F892F881FCC
:104C7000990BEB85FC858E0F9F1F90938502809387
:104C80008402EF85F8892B893C89E29FC001E39F6C
:104C9000900DF29F900D1124880F892F881F990B7A
:104CA000E989FA898E0F9F1F909383028093820275
:104CB000ED89FE89298D3A8DE29FC001E39F900D19
:104CC000F29F900D1124880F892F881F990BEF896F
:104CD000F88D8E0F9F1F9093810280938002EB8D41
:104CE000FC8D2F8D38A1E29FC001E39F900DF29FB4
:104CF000900D1124880F892F881F990BED8DFE8D43
:104D00008E0F9F1F90937F0280937E029501D601A4
:104D10000E9410353FE095958795779567953A9570
:104D2000D1F76E0D7F1D70937D0260937C02980118
:104D3000DA010E941035EFE0959587957795679594
:104D4000EA95D1F7E9A1FAA16E0F7F1F70937B025C
:104D500060937A0250937902409378025595479573
:104D600055954795405840938D02A2960FB6F894FA
:104D7000DEBF0FBECDBFDF91CF91FF91EF91BF910D
:104D8000AF919F918F917F916F915F914F913F91E3
:104D90002F911F910F91FF90EF90DF90CF90BF90D8
:104DA000AF909F908F907F906F905F904F903F90CB
:104DB0002F900F900FBE0F901F901895CF92DF92FB
:104DC000EF92FF920F931F93CF93DF936B017C01C0
:104DD000F7FE0FC062E079E286EA92E00E941E22AE
:104DE000F094E094D094C094C11CD11CE11CF11C3F
:104DF000EFCFC114D104E104F10419F466EE7EE2B0
:104E0000E6C088EEC81683E0D806E104F1042CF170
:104E1000C701B60128EE33E040E050E00E94EB34D9
:104E20008B01D82FC92FB901882777FD8095982F3E
:104E30000E94DE2669EA79E286EA92E00E941E225A
:104E40006801ED2EFC2ED701C6010197A109B10919
:104E500083369105A105B10520F184E6C816D10479
:104E6000E104F10424F1C701B60124E630E040E09A
:104E700050E00E94EB348B01D82FC92FCA01B90131
:104E80000E94DE2662E27AE286EA92E00E941E2218
:104E90006801ED2EFC2EC114D104E104F10409F4E3
:104EA000A2C062E579E286EA92E00E941E2284E1D5
:104EB000C816D104E104F1040CF441C0C701B601E5
:104EC0002AE030E040E050E00E94EB34C901AA271C
:104ED00097FDA095BA2FFC013397E730F10520F438
:104EE000EC5CFF4F0C940A3563EB7AE21AC06BE579
:104EF0007BE211C064ED7DE20EC065E37BE20BC096
:104F00006FE47DE208C065E07DE205C062ED7CE211
:104F100002C06AE77CE286EA92E00E941E2269E70C
:104F20007AE286EA92E00E941E22C701B6012AE0D8
:104F300030E040E050E00E94EB346B017C01F60170
:104F40003197E331F10508F04EC0E55CFF4F0C945A
:104F50000A3563EA7EE23BC06CE67EE238C060E27E
:104F60007EE235C064ED7DE232C061E87DE22FC0B3
:104F70006FE47DE22CC065E07DE229C062ED7CE259
:104F800026C06AE77CE223C064E47CE220C06CEDCA
:104F90007BE21DC063E97BE21AC06BE57BE211C0D6
:104FA00064ED7DE20EC065E37BE20BC06FE47DE261
:104FB00008C065E07DE205C062ED7CE202C06AE700
:104FC0007CE286EA92E00E941E226FEF7AE286EA95
:104FD00092E0DF91CF911F910F91FF90EF90DF90C2
:104FE000CF900C941E22DF91CF911F910F91FF90D3
:104FF000EF90DF90CF900895079731F461EB78E35D
:1050000086EA92E00C941E2208956A30710530F50C
:10501000FB01E25BFF4F0C940A3565E572E31AC0B1
:105020006FEE71E317C06CEB71E314C064E571E3DC
:1050300011C067EF70E30EC069E770E30BC066E470
:1050400070E308C06EEE7FE205C067EA7FE202C04F
:1050500063E37FE286EA92E00C941E22089581E0E9
:105060000E94C131BC01882777FD8095982F0E944E
:10507000B63320E030E040EA50E40E9442342AEAAD
:1050800031EF42E85FE30E941B330E94833388279D
:1050900077FD8095982F0E94DE2669EC78E286EAFB
:1050A00092E00E941E226CE878E286EA92E00C947C
:1050B0001E2281E00E94C131BC01882777FD8095C6
:1050C000982F0E94B63320E030E040EA50E40E947E
:1050D00042342AEA31EF42E85FE30E941B330E9428
:1050E0008333882777FD8095982F0E94DE2666E41B
:1050F00078E286EA92E00C941E228330910599F0C2
:1051000034F48130910549F0029751F008958430CC
:10511000910561F0059769F0089567E373E00BC0AE
:105120006DED72E008C063E872E005C06CE272E009
:1051300002C06CEC71E086EA92E00C941E220197AA
:105140008A31910508F056C0885A9F4FFC010C9493
:105150000A3563E872E44AC06BE272E447C069EC66
:1051600071E444C066E771E441C064E371E43EC0A9
:105170006FE970E43BC067E670E438C061EF7FE33D
:1051800035C061E97FE332C06BE27FE32FC06EED93
:105190007EE32CC06BE97EE329C069E57EE326C08F
:1051A0006DEB7DE323C060E67DE320C06EE17DE32F
:1051B0001DC067ED7CE31AC067E77CE317C061EEB2
:1051C0007BE314C06AE67BE311C06CEE7AE30EC0A9
:1051D00069E77AE30BC060E27AE308C06CEA79E33E
:1051E00005C069E479E302C060E079E386EA92E011
:1051F0000C941E220895AF92BF92CF92DF92EF924D
:10520000FF920F931F9381E00E94C131BC01882758
:1052100077FD8095982F1F921F921F922AE12F935E
:10522000A12CB12C6501A394EE24EA9413E0F12E95
:1052300000E010E020E030E0A9010E94D3320F909E
:105240000F900F900F90CB01AA2797FDA095BA2F32
:10525000FC013197EA31F10508F05DC0EE58FF4FCF
:105260000C940A3563E878E34AC061E578E347C007
:105270006FE078E344C06BED77E341C065EA77E324
:105280003EC06BE677E33BC06DE277E338C062EF88
:1052900076E335C060EB76E332C06EE276E32FC092
:1052A0006DEE75E32CC061E776E329C06EEA75E325
:1052B00026C06EE675E323C060E475E320C06AE0B3
:1052C00075E31DC066ED74E31AC06AEA74E317C0A3
:1052D0006AE774E314C060E474E311C062E074E34D
:1052E0000EC06EEA73E30BC068E473E308C06FE0BE
:1052F00073E305C06DEC72E302C061E972E386EA14
:1053000092E01F910F91FF90EF90DF90CF90BF90B0
:10531000AF900C941E221F910F91FF90EF90DF90A1
:10532000CF90BF90AF900895CF93DF93EC01BC0175
:1053300043E0769567954A95E1F761708CE00E94AD
:105340004032BE01769567957695679561708BE0E2
:105350000E944032BE017695679561708AE00E9496
:1053600040326C2F617089E0DF91CF910C94403214
:10537000AF92BF92CF92DF92EF92FF920F931F9363
:1053800080E00E94C131BC01882777FD8095982F6D
:105390001F921F921F922DE02F93A12CB12C65011B
:1053A00012EFE12E13E0F12E00E010E020E030E0FB
:1053B000A9010E94D3327093A5026093A4020F90BA
:1053C0000F900F900F906A30710514F061E001C0EA
:1053D00060E08DE00E9440328091A4029091A5028D
:1053E0006AE070E00E94B5341F910F91FF90EF903A
:1053F000DF90CF90BF90AF900C949429EAE7F0E053
:105400008081887F808380818560808361E08DE0FA
:105410000E94073261E089E00E94073261E08AE081
:105420000E94073261E08BE00E94073261E08CE06D
:105430000E94073262E085E00E94073262E084E069
:105440000E94073260E082E00E94073243E050E0B1
:1054500068EB79E280E00C946B30AF92BF92CF9210
:10546000DF92EF92FF920F931F9381E00E94C13170
:10547000BC01882777FD8095982F1F921F921F925D
:1054800029E02F93A12CB12C650118EEE12E13E039
:10549000F12E00E010E020E030E0A9010E94D332BC
:1054A0000F900F900F900F90882777FD8095982F81
:1054B0001F910F91FF90EF90DF90CF90BF90AF9032
:1054C0000C94DE2601978D30910508F0C5C08457F5
:1054D0009F4FFC010C940A3565E77CE086EA92E078
:1054E0000E941E226EE47CE086EA92E00E941E2268
:1054F00066ED7FE186EA92E00E941E2264ED7DE285
:1055000086EA92E00E941E226EE47CE086EA92E047
:105510000E941E226CEE7BE086EA92E00E941E2230
:1055200060EB7BE086EA92E00E941E226EE47CE063
:1055300086EA92E00E941E2263EA7EE289C06FE062
:1055400078E386EA92E00E941E2265E47BE086EA28
:1055500092E00E941E2266ED7AE07AC06CEE7BE05B
:1055600086EA92E00E941E226EE47CE086EA92E0E7
:105570000E941E2263E87AE06BC062E17AE086EA6C
:1055800092E00E941E226EE47CE041C064E779E074
:1055900086EA92E00E941E2268E279E086EA92E0C2
:1055A0000E941E226EE47CE086EA92E00E941E22A7
:1055B00065E47BE04DC06FEC78E032C06BED77E0E6
:1055C00086EA92E00E941E2264ED7DE286EA92E085
:1055D0000E941E2261EA77E03BC063E87AE086EA37
:1055E00092E00E941E226AE477E086EA92E00E943E
:1055F0001E226CEE76E02CC06AEA76E017C06CEBF7
:105600007CE086EA92E00E941E2262E576E086EA6D
:1056100092E00E941E2267EB79E01AC061EF75E00C
:1056200086EA92E00E941E226EE47CE086EA92E026
:105630000E941E2261E778E00BC06BE873E008C0AF
:1056400068E276E286EA92E00E941E226FE775E247
:1056500086EA92E00C941E22089581E00E94C131F6
:105660009093A00280939F0220919D0230919E0210
:10567000AC01421B530B9A0157FF03C03195219592
:1056800031092139314044F01092A2021092A10256
:1056900090939E0280939D026091A1027091A2025C
:1056A0006F5F7F4F7093A2026093A102882777FDFE
:1056B0008095982F0C94DE26CF93DF9381E00E9493
:1056C000C1319093A00280939F0220919D0230915E
:1056D0009E02821B930B97FF03C0919581959109C0
:1056E00081399140CCF16BEB7DE186EA92E00E943A
:1056F0001E2264E670E080E090E00E945E316BEE76
:105700007DE086EA92E00E941E2264EF71E080E074
:1057100090E00E945E31C3E0D0E06AE170E080E09A
:1057200090E00E94AF32CB010E949F2864E670E0B7
:1057300080E090E00E945E31219779F780919F028E
:105740009091A00290939E0280939D0264EF71E07D
:1057500080E090E00E945E31C4E0D0E069E070E05B
:1057600080E090E00E94AF320E94DE2664E670E0A6
:1057700080E090E00E945E31219781F764EF71E054
:1057800080E090E0DF91CF910C945E3181E00E9447
:10579000C1319093A00280939F0220919D0230918D
:1057A0009E02821B930B97FF03C0919581959109EF
:1057B000813991406CF060E070E0CB010E94992F3C
:1057C00080919F029091A00290939E0280939D02EF
:1057D0000E945B30BC01882777FD8095982F0E943E
:1057E000DE2665EA7DE086EA92E00E941E220E94A3
:1057F0006330BC01882777FD8095982F0E94DE26B4
:105800006BE37DE086EA92E00C941E22AF92BF9299
:10581000CF92DF92EF92FF920F931F9381E00E944D
:10582000C131BC01882777FD8095982F1F921F9268
:105830001F9229E02F93A12CB12C650118EEE12EC7
:1058400013E0F12E00E010E020E030E0A9010E941A
:10585000D3320F900F900F900F90882777FD80958F
:10586000982F1F910F91FF90EF90DF90CF90BF90F6
:10587000AF900C940528AF92BF92CF92DF92EF9237
:10588000FF920F931F9381E00E94C131BC018827D2
:1058900077FD8095982F1F921F9223E02F9327EE7C
:1058A0002F93A12CB12C6501EE24EA9413E0F12E84
:1058B00000E010E020E030E0A9010E94D3320F9018
:1058C0000F900F900F901F910F91FF90EF90DF902E
:1058D000CF90BF90AF900C94DE2601978E33910548
:1058E00008F0B9C087569F4FFC010C940A3566E159
:1058F00077E2ADC064E876E2AAC063E175E2A7C0D2
:105900006AEB74E2A4C069E574E2A1C065EC73E2DD
:105910009EC069E373E29BC06DEA72E298C06FE3D8
:1059200072E295C062ED71E292C06EE471E28FC0E6
:105930006AEC70E28CC06CE470E289C066ED7FE1D5
:1059400086C06CE57FE183C06BEF7EE180C06BE9D0
:105950007EE17DC061E47EE17AC06BEB7DE177C0E2
:1059600061E67DE174C06AEF7CE171C06BE77CE1C8
:105970006EC061ED7BE16BC064E67BE168C06EE008
:105980007AE165C06AE879E162C06FE279E15FC0FF
:105990006DEE78E15CC062E978E159C06FEF77E1C4
:1059A00056C068E377E153C06AEB76E150C066E029
:1059B00076E14DC066E77AE14AC06FE675E147C01F
:1059C0006AEC74E144C067E374E141C065EE73E1E1
:1059D0003EC06AE973E13BC06FE373E138C065EF35
:1059E00072E135C069E872E132C06BEB71E12FC042
:1059F00068E272E12CC064E071E129C066E570E103
:105A000026C067EB7FE023C068E77FE020C06DE041
:105A10007FE01DC066EA7EE01AC06BEE7DE017C035
:105A20006BE47EE014C065EA7DE011C06BE37DE0CD
:105A30000EC06CEB7CE00BC064E877E208C069EC58
:105A400077E205C068E276E202C06FE775E286EAB7
:105A500092E00C941E220895AF92BF92CF92DF92F3
:105A6000EF92FF920F931F930E94B8294C9B18C08E
:105A70008091A302813051F44A99FECF6AE070E030
:105A800080E090E00E945E311092A3020E94B8294B
:105A900082E00E947632892BC9F381E08093A302D1
:105AA000E091A402F091A502EF30F10508F03BC1AE
:105AB000E952FF4F0C940A351F910F91FF90EF9020
:105AC000DF90CF90BF90AF900C942D2A1F910F9133
:105AD000FF90EF90DF90CF90BF90AF900C94062C8A
:105AE0001F910F91FF90EF90DF90CF90BF90AF90FC
:105AF0000C94FB2881E00E94C131BC01882777FD0E
:105B00008095982F1F921F921F922AE12F93A12C0C
:105B1000B12C6501A39418EEE12E13E0F12E00E004
:105B200010E020E030E0A9010E94D3320F900F90E6
:105B30000F900F90CB011F910F91FF90EF90DF908E
:105B4000CF90BF90AF900C949F2881E00E94C1310C
:105B5000BC01882777FD8095982F1F921F921F9276
:105B60002EE32F93A12CB12C6501A394EE24EA948B
:105B700013E0F12E00E010E020E030E0A9010E94E7
:105B8000D3320F900F900F900F9042C01F910F9142
:105B9000FF90EF90DF90CF90BF90AF900C943B2C94
:105BA0001F910F91FF90EF90DF90CF90BF90AF903B
:105BB0000C942F281F910F91FF90EF90DF90CF90C2
:105BC000BF90AF900C9459281F910F91FF90EF90C8
:105BD000DF90CF90BF90AF900C942D2B1F910F9121
:105BE000FF90EF90DF90CF90BF90AF900C945C2B24
:105BF0001F910F91FF90EF90DF90CF90BF90AF90EB
:105C00000C94C62B6EE370E080E090E00E94AF320F
:105C1000CB011F910F91FF90EF90DF90CF90BF903D
:105C2000AF900C946D2C81E00E94C131BC0188279B
:105C300077FD8095982F1F921F921F922DE02F9332
:105C4000A12CB12C6501A394EE24EA9413E0F12E6B
:105C500000E010E020E030E0A9010E94D3320F9074
:105C60000F900F900F90CB011F910F91FF90EF902D
:105C7000DF90CF90BF90AF900C94622A81E00E9499
:105C8000C131BC01882777FD8095982F1F921F9204
:105C90001F9225E02F93A12CB12C6501A39412EF44
:105CA000E12E13E0F12E00E010E020E030E0A90149
:105CB0000E94D3320F900F900F900F90CB011F9145
:105CC0000F91FF90EF90DF90CF90BF90AF900C942A
:105CD0007D2881E00E94C131BC01882777FD809535
:105CE000982F1F921F921F9229E02F93A12CB12C65
:105CF000650115EFE12E13E0F12E00E010E020E049
:105D000030E0A9010E94D3320F900F900F900F90B6
:105D1000CB011F910F91FF90EF90DF90CF90BF903C
:105D2000AF900C94FC271F910F91FF90EF90DF90A4
:105D3000CF90BF90AF9008956F927F928F929F9275
:105D4000AF92BF92CF92DF92EF92FF920F931F9389
:105D5000CF93DF93EA012CE3C22ED12CE12CF12C5E
:105D6000A70196010E94C9346883CA01B901A7013D
:105D700096010E94C9346983CA01B90128E130E063
:105D800040E050E00E94C93449015A016A83CA01C7
:105D9000B9016C5F7F4F8F4F9F4F27E030E040E0AD
:105DA00050E00E94C9346F5F6B8300E010E09801FF
:105DB00040E054E6652E712C60E9C62EDD24D394B4
:105DC000E42FF0E0EE54F84F7F0183E0E822FF2457
:105DD000E114F10489F4CF01B3010E94B534892B99
:105DE00029F08EE691E0A0E0B0E00AC0CF01B60154
:105DF0000E94B534892BA9F38DE691E0A0E0B0E0D4
:105E0000080F191F2A1F3B1FD901C801AA27BB274A
:105E100088169906AA06BB0610F04F5FD1CF4E83B5
:105E2000E114F10499F4CF0164E670E00E94B53406
:105E3000892B29F08EE691E0A0E0B0E00BC0CF0105
:105E400060E971E00E94B534892BA1F38DE691E001
:105E5000A0E0B0E0081B190B2A0B3B0B801A910A3B
:105E6000A20AB30ACF0164E670E00E94B5349C0137
:105E7000CF0160E971E00E94B534ECE6F2E0A0E009
:105E8000A13059F4E114F10451F42115310511F058
:105E90004DE106C00097E1F302C0408101C04CE132
:105EA00050E060E070E084169506A606B70640F064
:105EB000841A950AA60AB70AAF5F3196AC3001F78B
:105EC000AF5FAD8383948C82DF91CF911F910F914F
:105ED000FF90EF90DF90CF90BF90AF909F908F900A
:105EE0007F906F900895CF92DF92EF92FF926B01B7
:105EF0007C018091BA029091BB02A091BC02B0914A
:105F0000BD02C816D906EA06FB0671F04EEB52E058
:105F1000C701B6010E949C2EC092BA02D092BB0269
:105F2000E092BC02F092BD02FF90EF90DF90CF9024
:105F300008950F931F936093B6027093B7028093F6
:105F4000B8029093B9020091670210916802209103
:105F5000690230916A02060F171F281F391F00932C
:105F6000AE021093AF022093B0023093B10282E0F0
:105F700090E09093AD028093AC020E942F31609329
:105F8000B2027093B3028093B4029093B5021F9152
:105F90000F910895CF92DF92EF92FF920F931F938C
:105FA0000E942F31C090B202D090B302E090B402B0
:105FB000F090B5026C197D098E099F090091B60217
:105FC0001091B7022091B8023091B902683E734037
:105FD00081059105D8F00F5F1F4F2F4F3F4F009362
:105FE000B6021093B7022093B8023093B90248EE7C
:105FF000C40E43E0D41EE11CF11CC092B202D09248
:10600000B302E092B402F092B502CACF8091AE0220
:106010009091AF02A091B002B091B1020817190798
:106020002A073B07C8F1E091AA02F091AB02309732
:1060300099F10995611571058105910519F00E9485
:10604000992F2AC08091670290916802A0916902FD
:10605000B0916A024091B6025091B7026091B802C5
:106060007091B902840F951FA61FB71F8093AE02CF
:106070009093AF02A093B002B093B10281E090E0A0
:106080002091AC023091AD02232B11F480E090E01E
:106090009093AD028093AC026091B6027091B7020A
:1060A0008091B8029091B9021F910F91FF90EF90EB
:1060B000DF90CF9008950E94CA2F0E94732F809185
:1060C000BF0290E008950E94CA2F0E94732F809112
:1060D000BE0290E008958230E8F4E82FF0E0EE0F81
:1060E000FF1FEB53FD4F71836083813041F080913E
:1060F00069008C7F842B80936900E89A08958091D1
:106100006900440F551F440F551F837F842B8093D4
:106110006900E99A08951F920F920FB60F92112409
:106120002F933F934F935F936F937F938F939F939F
:10613000AF93BF93EF93FF938091C5029091C602F6
:10614000892B29F0E091C502F091C6020995FF91D3
:10615000EF91BF91AF919F918F917F916F915F91DF
:106160004F913F912F910F900FBE0F901F90189558
:106170001F920F920FB60F9211242F933F934F93BC
:106180005F936F937F938F939F93AF93BF93EF939F
:10619000FF938091C7029091C802892B29F0E0916A
:1061A000C702F091C8020995FF91EF91BF91AF919D
:1061B0009F918F917F916F915F914F913F912F911F
:1061C0000F900FBE0F901F9018951F920F920FB651
:1061D0000F9211242F933F938F939F93AF93BF936D
:1061E0008091CA029091CB02A091CC02B091CD02D5
:1061F0003091C90223E0230F2D3720F40196A11D11
:10620000B11D05C026E8230F0296A11DB11D2093E4
:10621000C9028093CA029093CB02A093CC02B093A0
:10622000CD028091CE029091CF02A091D002B09188
:10623000D1020196A11DB11D8093CE029093CF0291
:10624000A093D002B093D102BF91AF919F918F9153
:106250003F912F910F900FBE0F901F9018952FB761
:10626000F8946091CA027091CB028091CC02909117
:10627000CD022FBF08953FB7F8948091CE02909140
:10628000CF02A091D002B091D10226B5A89B05C043
:106290002F3F19F00196A11DB11D3FBF6627782F32
:1062A000892F9A2F620F711D811D911D42E0660F8B
:1062B000771F881F991F4A95D1F70895CF92DF92D3
:1062C000EF92FF92CF93DF936B017C010E943B31F1
:1062D000EB01C114D104E104F10489F00E941A33E6
:1062E0000E943B316C1B7D0B683E734090F381E054
:1062F000C81AD108E108F108C851DC4FEACFDF9194
:10630000CF91FF90EF90DF90CF900895789484B56F
:10631000826084BD84B5816084BD85B5826085BDA1
:1063200085B5816085BDEEE6F0E080818160808387
:10633000E1E8F0E01082808182608083808181606A
:106340008083E0E8F0E0808181608083E1EBF0E031
:10635000808184608083E0EBF0E0808181608083D5
:10636000EAE7F0E0808184608083808182608083BE
:106370008081816080838081806880831092C100E9
:1063800008958E3008F08E50877020916B0290E453
:10639000299F90011124822B80937C0080917A00A8
:1063A000806480937A0080917A0086FDFCCF809192
:1063B00078002091790090E0922B0895833081F04D
:1063C00028F4813099F08230A1F008958630A9F048
:1063D0008730B9F08430D1F4809180008F7D03C084
:1063E000809180008F7780938000089584B58F77A7
:1063F00002C084B58F7D84BD08958091B0008F77F1
:1064000003C08091B0008F7D8093B0000895CF933A
:10641000DF9390E0FC01E550FD4B2491FC01E15F2E
:10642000FC4B8491882349F190E0880F991FFC016F
:10643000E95CFC4BA591B491835D9C4BFC01C5913B
:10644000D4919FB7611108C0F8948C912095822354
:106450008C93888182230AC0623051F4F8948C9125
:10646000322F309583238C938881822B888304C0BC
:10647000F8948C91822B8C939FBFDF91CF910895DC
:106480000F931F93CF93DF931F92CDB7DEB7282FC3
:1064900030E0F901E951FD4B8491F901E550FD4BE4
:1064A0001491F901E15FFC4B04910023C9F08823AA
:1064B00021F069830E94DE316981E02FF0E0EE0F68
:1064C000FF1FE35DFC4BA591B4919FB7F8948C91AD
:1064D000611103C01095812301C0812B8C939FBF54
:1064E0000F90DF91CF911F910F910895CF93DF937C
:1064F000282F30E0F901E951FD4B8491F901E55075
:10650000FD4BD491F901E15FFC4BC491CC2391F098
:1065100081110E94DE31EC2FF0E0EE0FFF1FED5DE8
:10652000FC4BA591B4912C912D2381E090E021F4B6
:1065300080E002C080E090E0DF91CF91089508955F
:106540000E9486310E949F320E94FE29C0E0D0E066
:106550000E942C2D2097E1F30E940000F9CFCF93E9
:10656000DF9300D000D0CDB7DEB79B01AC01611541
:1065700071058105910569F069833A834B835C83DA
:106580000E94A43529813A814B815C810E94EB34C1
:1065900003C060E070E0CB010F900F900F900F9060
:1065A000DF91CF9108954F925F926F927F92AF9259
:1065B000BF92CF92DF92EF92FF920F931F93CF93F0
:1065C000DF93CDB7DEB729013A01621B730B840B51
:1065D000950B29893A894B895C892A193B094C0911
:1065E0005D09298B3A8B4B8B5C8B9B01AC016989D4
:1065F0007A898B899C890E94A534E418F5080609DC
:106600001709A80197010E94EB342A0D3B1D4C1D70
:106610005D1DCA01B901DF91CF911F910F91FF90CC
:10662000EF90DF90CF90BF90AF907F906F905F9092
:106630004F90089508950CD0EBC0E3D040F0DAD02D
:1066400030F021F45F3F19F0CCC0511115C1CFC01B
:10665000F0D098F39923C9F35523B1F3951B550B4B
:10666000BB27AA2762177307840738F09F5F5F4F25
:10667000220F331F441FAA1FA9F333D00E2E3AF066
:10668000E0E830D091505040E695001CCAF729D080
:10669000FE2F27D0660F771F881FBB1F26173707CF
:1066A0004807AB07B0E809F0BB0B802DBF01FF27FF
:1066B00093585F4F2AF09E3F510568F092C0DCC0AE
:1066C0005F3FECF3983EDCF3869577956795B79539
:1066D000F7959F5FC9F7880F911D9695879597F954
:1066E0000895E1E0660F771F881FBB1F62177307CD
:1066F0008407BA0720F0621B730B840BBA0BEE1FE2
:1067000088F7E095089504D06894B111B5C0089554
:1067100098D088F09F5790F0B92F9927B751A0F0E3
:10672000D1F0660F771F881F991F1AF0BA95C9F725
:1067300012C0B13081F09FD0B1E008959CC0672FA6
:10674000782F8827B85F39F0B93FCCF386957795D5
:106750006795B395D9F73EF49095809570956195BE
:106760007F4F8F4F9F4F0895E89409C097FB3EF4E9
:1067700090958095709561957F4F8F4F9F4F99238E
:10678000A9F0F92F96E9BB279395F695879577950C
:106790006795B795F111F8CFFAF4BB0F11F460FFCC
:1067A0001BC06F5F7F4F8F4F9F4F16C0882311F024
:1067B00096E911C0772321F09EE8872F762F05C038
:1067C000662371F096E8862F70E060E02AF09A95D3
:1067D000660F771F881FDAF7880F9695879597F9C8
:1067E000089597F99F6780E870E060E008959FEF53
:1067F00080EC089500240A94161617061806090658
:10680000089500240A941216130614060506089526
:10681000092E0394000C11F4882352F0BB0F40F4AE
:10682000BF2B11F460FF04C06F5F7F4F8F4F9F4FEE
:10683000089557FD9058440F551F59F05F3F71F070
:106840004795880F97FB991F61F09F3F79F08795D7
:106850000895121613061406551FF2CF4695F1DF60
:1068600008C0161617061806991FF1CF86957105F0
:10687000610508940895E894BB2766277727CB0124
:1068800097F908950BD0C4CFB5DF28F0BADF18F020
:10689000952309F0A6CFABCF1124EECFCADFA0F32A
:1068A000959FD1F3950F50E0551F629FF001729FA5
:1068B000BB27F00DB11D639FAA27F00DB11DAA1FC4
:1068C000649F6627B00DA11D661F829F2227B00D11
:1068D000A11D621F739FB00DA11D621F839FA00D9C
:1068E000611D221F749F3327A00D611D231F849FEC
:1068F000600D211D822F762F6A2F11249F57504043
:106900008AF0E1F088234AF0EE0FFF1FBB1F661FDD
:10691000771F881F91505040A9F79E3F510570F096
:1069200060CFAACF5F3FECF3983EDCF38695779576
:106930006795B795F795E7959F5FC1F7FE2B880F91
:10694000911D9695879597F90895DB018F939F93F5
:106950000E942E35BF91AF91A29F800D911DA39FE4
:10696000900DB29F900D1124089597FB072E16F4F9
:10697000009407D077FD09D00E94413507FC05D06F
:106980003EF4909581959F4F0895709561957F4F46
:106990000895A1E21A2EAA1BBB1BFD010DC0AA1F60
:1069A000BB1FEE1FFF1FA217B307E407F50720F078
:1069B000A21BB30BE40BF50B661F771F881F991FF3
:1069C0001A9469F760957095809590959B01AC013C
:1069D000BD01CF010895052E97FB1EF400940E947F
:1069E000023557FD07D00E94C93407FC03D04EF48E
:1069F0000C94023550954095309521953F4F4F4F5F
:106A00005F4F089590958095709561957F4F8F4F5A
:106A10009F4F0895EE0FFF1F0590F491E02D09940C
:106A20000E941835332312F48A1B9B0B0C942935D2
:106A3000A29FB001B39FC001A39F700D811D1124BF
:106A4000911DB29F700D811D1124911D08950E940A
:106A50001835B7FF0895821B930B08950E941835CF
:106A6000A59F900DB49F900DA49F800D911D1124A2
:106A70000895B7FF0C942E350E942E35821B930B80
:106A80000895AA1BBB1B51E107C0AA1FBB1FA61775
:106A9000B70710F0A61BB70B881F991F5A95A9F7C7
:106AA00080959095BC01CD0108958F929F92AF92F1
:106AB000BF92CF92DF92EF92FF92CF93DF93EC01E0
:106AC000688179818A819B816115710581059105B4
:106AD00021F464E279ED8BE597E02DE133EF41E0BD
:106AE00050E00E94EB3449015A019B01AC01A7EA36
:106AF000B1E40E942E356B017C01ACEEB4EFA50130
:106B000094010E943C35C60ED71EE81EF91EF7FE02
:106B100006C081E0C81AD108E10880E8F80AC882F6
:106B2000D982EA82FB82C701B6019F77DF91CF91BC
:106B3000FF90EF90DF90CF90BF90AF909F908F909D
:106B400008950E945535089580E091E00E945535E2
:106B50000895609300017093010180930201909366
:086B600003010895F894FFCF32
:106B6800010000000100002AD432B212251402E10B
:106B7800C5025F5A050F26FCA5A5D6DDDCFC252B32
:106B880022210FFFF8EEEDEFF7F6FA00030201CD30
:106B9800DFF10416203B4DC0D4E8FC1025394DC068
:106BA800D8F0071F374F66B3BFCBD7E3EFFB071308
:106BB8001F2B37434F5A66C0CBD6E1ECF7030E19AB
:106BC800242F3A45505B66AEBAC5D1DDE8F4FF0B19
:106BD80017222E3945515CAEBCCAD8E6F4010F1D08
:106BE8002B39475563717E929FADBAC8D5E3F0FE45
:106BF8000B192634414F5C00AE80B480BB40C38083
:106C0800CB40D4C0DD80E780F1C0FB0006401040D7
:106C18001A0024402D0036403EC045C04C00538029
:106C280058C05D40624066C069C06C806FC071C06A
:106C38007380750077807EC0828083C0834084C063
:106C48008440850086808780888089C08A008C403F
:106C58008D008FC090C092009940A180AB40B84091
:106C6800C7C0D8C0EB000040144027C038C04780D8
:106C780054C05E0067406D001011121314151617EA
:106C880018191A1B1C1D1E1F202122232425262704
:106C980028292A2B2D2F31333536393B3D3F4245A4
:106CA80047494D4F5155575C5F63666A6E73777BF2
:106CB80080858A8F959AA00002030405070A0F149D
:106CC8002029395172A1FF2C010000011F1C1F1E31
:086CD8001F1E1F1F1E1F1E1FBF
:00000001FF
